:10400000008000208FC8000045C8000047C800009D
:1040100000000000000000000000000000000000A0
:1040200000000000000000000000000049C800007F
:1040300000000000000000004BC8000009860000DE
:104040004FC8000051C8000053C8000055C8000008
:1040500057C8000009A600005BC800005DC800004A
:104060005FC80000D9A6000063C8000065C8000052
:1040700067C8000069C800006BC80000E981000043
:104080006FC8000071C8000073C8000075C8000048
:1040900077C8000079C800007BC800007DC8000018
:1040A0007FC8000081C80000D140000085C8000022
:1040B00087C8000089C800008BC800008DC80000B8
:0840C000FFFFFFFFFFFFFFFF00
:1040C80062B6704772B6704708B506F0CFFF08BDF4
:1040D80073B5314B314C01226260A260E361304B11
:1040E80030492362202323638023DB00E3623823E3
:1040F8008B60E0202C4B40035A609A6018622B4872
:10410800D861C0200001D862C02080001863C02395
:104118001B048B61101C152108F004F900230A21E7
:104128001A1C0420E0620120206300200190019DF8
:104138001F48854202D801980130F7E7A56BAE0603
:1041480006D5164DAE6B082535406E42754152199D
:104158000125E5620425256300250195019D854219
:1041680002D8019D0135F8E7A06B850604D40B48F9
:10417800806B0007C00F1B1801390029D1D1052118
:1041880021630C490A2A03D10A2B01D1012300E03B
:1041980000230B7073BDC0460704000000000540F3
:1041A800380000C00080054000100540E00F4000C6
:1041B800E70300006808002000B5072819D808F0B0
:1041C80085FB04070B0D0F1113158022520001E027
:1041D80080229200074B0BE0042208E0022206E04E
:1041E800012204E0202202E0102200E00822024B13
:1041F800DA6200BD001005400000054000B5072840
:1042080019D808F063FB04070B0D0F111315802252
:10421800520001E080229200074B0BE0042208E0E4
:10422800022206E0012204E0202202E0102200E03F
:104238000822024B1A6300BD00100540000005402B
:1042480008B50023062826D808F040FB040C1015F2
:10425800191D2100002006F031FA104B83429B41C2
:104268005B4218E00E4B9B6B9B0602E00C4B9B6B72
:10427800DB06DB0F0FE00A4B9B6B1B07F9E7084BCC
:104288009B6B5B07F5E7064B9B6B9B07F1E7044BC2
:104298009A6B01231340181C08BDC046FF03000099
:1042A8000000054000B50023072825D8012208F0A2
:1042B8000DFB04080C1014171B1F104B5B6B1B0A1B
:1042C80019E00E4B5B6B5B0A15E00D4B5B6B9B08B3
:1042D80011E00B4B5B6B5B080DE0094B5B6B0AE075
:1042E800074B5B6B5B0906E0054B5B6B1B0902E048
:1042F800034B5B6BDB081340181C00BD0010054026
:1043080000000540124B0422C10701D5DA6100E024
:104318001A620222104201D0DA6100E01A62012218
:10432800410701D5DA6100E01A622022010701D5B0
:10433800DA6100E01A621022104201D0DA6100E06E
:104348001A620822810601D5DA6100E01A62704714
:1043580000000540144910B58B680422C40701D534
:10436800134300E093430222104201D0134300E0BC
:1043780093430122440701D5134300E093432022CD
:10438800040701D5134300E093431022104201D0E3
:10439800134300E093430822840601D5134300E049
:1043A80093438B6010BDC0460080054062B67047DD
:1043B80072B6704708B5002802D008F011F901E07C
:1043C80008F016F908BD08B5002802D1C90804F09C
:1043D8000FFD08BD031C0020834203D1024B986BDC
:1043E800C002C00F7047C04600100540104B82B095
:1043F8001B78002B19D00F4B8022DA6240221A63F7
:104408000022019201990C4A914202D8019A013284
:10441800F7E7802119634021D96200230193019BAA
:104428009342E8D8019B0133F8E702B07047C046D1
:1044380068080020001005409F86010008B500208C
:104448000721012207F06EFF00200821012207F052
:1044580069FF00200921012207F064FF01200E21D5
:10446800032207F05FFF01200D21032207F05AFF06
:1044780001200C21032207F055FF0A4B8022D200AD
:10448800DA62094BC0221201DA62084B0222C72104
:10449800082019605A601861054B19605A60282273
:1044A8001A6108BD000005400010054000000940E1
:1044B8000010094001280DD0002808D0022825D175
:1044C800134B8020C0001863124B99600DE08020C8
:1044D800000101E08020C0000F4B18630F4B99606A
:1044E800D968C806FCD40D4B03E0D968C806FCD4CB
:1044F800084B9868C0B2002A09D0074BC0221201A5
:10450800DA628022024BD200DA6200E000207047B3
:104518000000054000000940001005400010094057
:1045280073B5A54C63789A1F012A0ED98C2B0CD031
:10453800C02B0AD0C72B08D06632D2B2182A04D9A9
:104548001A1C3432D2B2322A04D8A278002A04D0F3
:10455800042225E3A278022AFAD8A42B00D190E2FB
:1045680000D984E0842B00D12CE128D8062B00D177
:1045780095E110D8022B00D124E106D8002B00D1F8
:1045880004E1012B00D104E109E3042B00D147E148
:1045980000D841E168E1802B00D1F7E009D80C2B65
:1045A80000D18AE10D2B00D19DE1072B00D0F6E266
:1045B8007CE1822B00D1ACE100D8EAE030E1942B19
:1045C80000D17AE126D88A2B00D1B5E10BD8862B09
:1045D80000D149E100D21FE1872B00D0DFE2A178AA
:1045E8000E23490198E18D2B00D1BAE1932B00D11C
:1045F80079E18C2B00D0D2E2E3780821C91AA0789F
:10460800C9B204F0B1FAA3786C4A5B01D318E27816
:10461800DA72C7E2A02B00D124E21ED8992B00D170
:10462800B0E19A2B00D1BEE1952B00D0B7E2A1787A
:1046380014234901194301ADC9B22A1C002005F011
:104648001BFD2179E37809021943637904221B04CD
:104658001943A3791B06194387E1A22B00D106E26F
:1046680000D909E2A078E17804F09EFA9AE2B32B27
:1046780000D13EE23AD8AB2B00D11BE218D8A72BC9
:1046880000D108E20AD8A52B00D1FFE1A62B00D063
:1046980085E2A078E17804F0DBFA83E2A92B00D167
:1046A800FEE100D901E2A078E17804F01DFB79E28F
:1046B800AF2B00D10EE20FD8AD2B00D1FFE100D90E
:1046C80002E2E178A07804F03FFBA3783C49DB00E4
:1046D800E278CB185A7165E2B12B00D1FFE100D91D
:1046E80002E2A078E17804F0B7FB5BE2C32B00D1CB
:1046F80081E124D8B82B00D11CE217D8B62B00D101
:10470800FCE100D90FE2B52B00D048E2A3782B4A90
:104718005B01D3182279E17812020A43617909040E
:104728000A43A17909060A439A613BE2C12B00D1E9
:104738004BE100D950E1C02B00D1B7E02FE2D22BDA
:1047480000D10AE209D8CC2B00D164E1D12B00D1E9
:10475800F5E1C72B00D022E2A1E0D62B00D164E11D
:10476800FE2B00D16BE1D42B00D018E2A378134ABA
:104778005B01D3182279E17812020A4361790904AE
:104788000A43A17909060A435A610BE2A178490153
:1047980003E0A1780223490119432279E378120240
:1047A8001A436379C9B21B041A43A37900201B0674
:1047B8001A4305F0D1FBF5E1DC020020C80800200F
:1047C8003C080020A1780823227949011943E3789D
:1047D80012021A436379C9B21B041A43A379002051
:1047E8001B061A4305F0AAFBA17806232279490182
:1047F8001943E37812021A436379C9B21B041A43B6
:10480800A37900201B061A43D317D2185A4005F083
:1048180095FBA378012124E0A1780A2349017BE0D4
:10482800A1780623227949011943E37812021A4331
:104838006379C9B21B041A43A37900201B061A43E3
:1048480005F07CFB2079E278000210436279A378B6
:1048580012041043A279990012061043D24A8850D4
:104868000021D24AD1549DE12179E3780902194304
:104878006379A0781B041943A3791B06194305F033
:1048880072FC2079E278000210436279A37812045E
:104898001043A279990012061043C54ADFE7A378AE
:1048A800C44A5B01D318E2785A727BE1A378C14A03
:1048B8005B01D318E2789A7274E1A1781423490154
:1048C800194301ADC9B22A1C002005F0D5FB217996
:1048D800E37809021943637902221B041943A37977
:1048E8001B06194341E0A17814234901194301AD7E
:1048F800C9B22A1C002005F0BFFB2179E378090220
:104908001943637901221B041943A3791B06194330
:104918002BE0A1780423490122791943E378120294
:104928001A436379C9B21B041A43A37900201B06F2
:104938001A4305F003FB35E1A1781426490101ADBE
:104948003143C9B200202A1C05F096FBE378AB700E
:10495800A17849010E43F1B200202A1C05F0D2FAD1
:1049680020E1A1781A234901D6E76B78002901D004
:10497800134300E093436B70A17814234901194352
:10498800C9B2E9E7A1781826490101AD3143C9B296
:104998002A1C002005F070FB69780F23E278994300
:1049A8001A400B1C0EE0A1781826490101AD3143CD
:1049B800C9B22A1C002005F05FFBE27869780F2352
:1049C80012010B4013436B70C2E7A378794A5B016D
:1049D800D318E2781A72E5E02179E37809021943DD
:1049E8006379A2781B041943A37952011B06194362
:1049F800704BD150D6E0A3786E4A5B01D318227968
:104A0800E17812020A43617909040A43A179090687
:104A18000A435A60C6E0A378664A5B01D318227934
:104A2800E17812020A43DA81BCE0A378614A5B01AB
:104A3800D3182279E17812020A439A83B2E02379E3
:104A4800E2781B0213436279A17812041343A27916
:104A5800490112061343574A5218002B00D001236C
:104A680013739FE0A078E17804F08EF89AE0A078BC
:104A7800E17804F0BBF895E0A078E17804F0C0F89C
:104A880090E0A078E17804F0CFF88BE0A078E178A6
:104A980004F0D4F886E0A078E17804F0E3F881E047
:104AA800A078E17804F02CF97CE0A078E17804F0B3
:104AB80033F977E0A078E17804F03AF972E0A07869
:104AC800E17804F07DF96DE00321A078615604F0E7
:104AD80083F967E0A078E17804F0B2F962E0A078A1
:104AE800E17804F0C5F95DE0A078E17804F0CCF94C
:104AF80058E0A078E17804F0DFF953E02279E37810
:104B080012021A436379A0781B041A43A3792A492D
:104B18001B061A43C3005A50002A43D1CB185979AF
:104B280004F012F93EE0A3782349DB00E278CB18C1
:104B38001A7137E0A078E17804F06CF832E0217956
:104B4800E378090219436379A0781B041943A37910
:104B58001B06194305F020FE24E0A078154A4301FE
:104B68002179D2186579E378090219432D0429437C
:104B7800A5792D06294311611F21194005F0D4FD9F
:104B88002179E378090219436379A0781B04194352
:104B9800A3791B061943491105F0BEFD02E0032263
:104BA800064B1A7073BDC04610080020580000203C
:104BB80004040020C80800203C080020F803002056
:104BC80073B5A24DA24C6B789A1F012A0ED98C2B73
:104BD8000CD0C02B0AD0C72B08D06632D2B2182A04
:104BE80004D91A1C3432D2B2322A05D8AA78002A3B
:104BF80005D00423237083E2AA78022AF9D8A32BCC
:104C080000D117E200D997E0832B00D150E13AD8C0
:104C1800082B00D160E115D8032B00D13FE105D85E
:104C2800012B00D12DE100D828E134E1052B00D17A
:104C380042E100D23CE1062B00D141E1072B00D133
:104C480044E149E20C2B00D14FE10AD80A2B00D1EC
:104C580075E100D963E10020FFF7F2FA431E98419D
:104C680017E1802B00D109E103D80D2B00D149E1D0
:104C780032E2812B00D104E1822B00D02CE2A9780A
:104C8800042349010EE1942B00D12EE123D8872B70
:104C980000D161E105D8852B00D100E100D8FAE008
:104CA8000AE18C2B00D15BE10ED88A2B00D013E2ED
:104CB800A97814234901194301ADC9B200202A1C5F
:104CC80005F0DAF9AB785BE18D2B00D153E1932B3A
:104CD80000D117E100E29C2B00D130E11AD8992BC2
:104CE80000D14FE10FD8952B00D0F5E1A978142316
:104CF8004901194301ADC9B200202A1C05F0BCF9CD
:104D08006B785B073BE19A2B00D149E19B2B00D1E3
:104D180005E1E1E1A02B00D184E103D89D2B00D16E
:104D2800DAE0D9E1A12B00D180E1A22B00D0D3E1B8
:104D3800A87803F0A1FFACE0B52B00D1B6E13AD8D2
:104D4800AC2B00D192E11BD8A72B00D17EE108D86B
:104D5800A52B00D172E100D974E1A87803F0A4FF73
:104D680097E0A92B00D179E100D273E1AA2B00D1F9
:104D780078E1AB2B00D0AFE1A87804F00DF888E01B
:104D8800B02B00D180E108D8AE2B00D174E100D956
:104D980076E1A87804F038F87BE0B22B00D17BE10B
:104DA80000D275E1B32B00D17AE1B42B00D093E1A6
:104DB800AB78284A78E1C72B00D181E01ED8C02BF8
:104DC80000D183E00BD8B72B00D17BE100D273E18F
:104DD800B82B00D080E1A87803F05EFF59E0C22B21
:104DE80000D1F0E000D2E8E0C32B00D1EFE0C42B03
:104DF80000D071E1AA78184B920060E1D12B00D164
:104E080066E115D8CE2B00D1E7E008D8CC2B00D02E
:104E180062E1AB78114A5B01D318DB89B0E0CF2B94
:104E280000D1DEE0D02B00D056E1AB780C4A3BE154
:104E3800D42B00D1EAE015D8D22B00D04CE1AB78C6
:104E4800064A5B01D3181B699AE0C046DC020020C1
:104E5800F80300203808002024080020C808002093
:104E6800C3080020D62B00D1D6E0FE2B00D033E1BA
:104E7800AB78A44A5B01D3181B7B81E0A978490170
:104E880003E0A978022349011943C9B2002005F0BB
:104E9800DFFA606022E1A9780823490102E0A978D5
:104EA8000A2349011943C9B2002005F0F7F8F0E7D1
:104EB800AA78954B920002E1AA78944B9200FEE002
:104EC800AB78904A5B01D3185B7A59E0AB788D4A8E
:104ED8005B01D3189B7A53E0002005F0C6F8AB7845
:104EE8005B00184101231840D3E7A978142349012E
:104EF800194301ADC9B200202A1C05F0BDF86B7832
:104F08009B073CE0A97814234901194301AD2A1CE9
:104F1800C9B2002005F0B0F86A7801233EE001AE7E
:104F2800321C00207C2105F0A7F8AB7802225B0038
:104F38009A40131CB27813405A1E934120E001AEE8
:104F4800321C00207C2105F097F8AB78B2785B0022
:104F58001A41131C012221E0A9780E234901A1E777
:104F6800AB78002B05D1002003F028FE0823181A7F
:104F78008FE70423B1E0A9781A23490192E7DB0FF0
:104F88006360ABE0A97818234901194301AD2A1CD5
:104F9800C9B2002005F070F86A780F231340EFE7D4
:104FA800A97818234901194301ADC9B200202A1C68
:104FB80005F062F86B781B09E2E7AB78514A5B01B0
:104FC800D3181B7ADCE7AA784E4B520177E0AB780E
:104FD8004C4A5B01D3185B68D2E7AA784C4B920025
:104FE8006DE000216160AB784A4AD05C884201D00C
:104FF80001206060D154484AD15C002903D0606820
:105008000221014361600021D15467E0AB783D4A39
:105018005B01D3185B69B3E7AB783A4A5B01D318F5
:105028009B8BADE7A87803F0D1FD32E7A87803F0B1
:10503800D5FD2EE7A87803F027FE2AE7A87803F025
:105048003BFE26E7A87803F03FFE22E7A87803F0A6
:1050580043FE1EE7A87803F083FE1AE7A87803F05A
:1050680087FE16E7A87803F08DFE12E7AB782B4A87
:10507800DB00D3185B7983E7A87803F0CDFE08E757
:10508800A87803F031FF04E7A87803F037FF00E7BA
:10509800A87803F03DFFFCE6A87803F043FFF8E6A4
:1050A800A87803F053FFF4E6D35C69E7AB78154AB8
:1050B8005B01D3189B6963E7AA78184BD200D258D2
:1050C80062600BE0AB78154ADB00D3181B7957E711
:1050D800A87805F053FBDCE603232370104B1B78FC
:1050E800002B0DD00F4B6168082219600E4B002968
:1050F80002D119680A4302E018689043021C1A603A
:1051080073BDC046C8080020100800200404002011
:105118005C080020C0080020570800203C08002038
:10512800F3030020E4030020E402002038B5CE4A4F
:105138009378141C022B00D186E1032B00D1A3E144
:10514800002B00D0E5E253784E2B00D1CFE052D8A7
:10515800452B00D19DE023D8422B00D18DE00AD801
:10516800402B00D186E0412B00D0D0E2D178BF4B54
:105178000020197085E0432B00D185E0442B00D036
:10518800C5E22379D2781B0213436279B749120426
:105198001343A2791C31120613430B601C208BE0C9
:1051A800492B00D18CE014D8462B77D0472B00D060
:1051B800ADE22379D2781B0213436279AB4D120416
:1051C8001343A279291C12061343AB600831082047
:1051D800CEE04C2B00D180E000D983E04B2B00D0EF
:1051E80095E2A24CD1780320E17002F047FEE07806
:1051F80003F0B6F890E2542B00D1C2E024D8512B2A
:1052080000D197E00AD84F2B00D183E0502B00D073
:105218007DE2D178954B1620997532E0522B00D15A
:1052280097E0532B00D072E22379D2781B02134304
:1052380062798E4D12041343A279291C1206134376
:105248002B611031102093E0832B00D1D5E006D8D4
:10525800552B00D1A7E0562B00D1B7E057E2852B9C
:1052680000D1E4E000D2D5E0FF2B00D04FE2D278A5
:105278007F4B50E2D1787F4803E0D1787B4B012007
:10528800597002F0FBFD47E2D178784B0420197180
:10529800F7E7D178754B05205971F2E72379D27871
:1052A8001B0213436279714912041343A2790C312A
:1052B800120613430B600C20042202F04BFE2BE273
:1052C800D2786A4B002A01D1DA7503E06A490122D3
:1052D800DA754A60D97D1720D3E7D178634B02206D
:1052E8009970CEE7D178614B15205975C9E71079C7
:1052F800D3780002184353795C4C1B041843937904
:105308001B061843E084FEF7FDFF211C26312620EA
:105318000222D2E7D178554C1920617602F0AEFD11
:10532800617E01231940081E01D00020191C05F0D8
:10533800C9F8F1E14D4A0123117D151C194204D029
:10534800E2781A4201D102F0F3FCE17814202975C1
:1053580097E72379D2781B021343627943491204F1
:105368001343A2792031120613430B602020A3E7D0
:10537800042202F0EFFD6879A9682A6903F000F8B1
:10538800CAE11179D3785079090292791943000456
:10539800014312060A43012A00D9BAE133491A2007
:1053A8008B761A3110E0D3781279617912020904E8
:1053B8001A430A43A17909060A43012A00D9A8E138
:1053C8002A491B20CB761B31012276E71379D17845
:1053D80052791B0212040B431343A279120613439A
:1053E8000F2B00D995E1002004F0A4FE1F49E278B4
:1053F8004B1DDA7724312420E6E71379D1781B0294
:105408000B435179927909040B4312061A431B4B3B
:105418005A6081E1D378127912021A4363791B0426
:105428001A43A3791B061A43154B1A6074E1D37803
:10543800127912021A4363791B041A43A3791B06D3
:105448001A430E4B9A6067E11379D0781B02034325
:105458005079517892790004034312061A43094B94
:105468008900CA5058E1C046DC020020080000202C
:10547800F2030020FF070000F80300205800002076
:10548800F40300201004002050782E2800D93EE1B3
:1054980007F026FA2F00400051003D013D013D0173
:1054A8003D013D013D0162006F007C003D013D0171
:1054B8003D013D013D013D013D013D013D013D01F4
:1054C8003D013D013D013D013D0189009500A100DF
:1054D800AD00B900C7003D013D013D013D013D0161
:1054E8003D01D500E200EF00FC000901160123018F
:1054F8003001D378127912021A4363791B041A43D4
:10550800A3791B061A43854B1A6003F0FDF8844BF8
:10551800D86001E1D378127912021A4363791B0427
:105528001A43A3791B061A437C4B5A6003F0ECF824
:105538007B4B1861F0E0D378127912021A43637931
:105548001B041A43A3791B061A43744B9A6003F091
:10555800DBF8734B5861DFE0D378127912021A43F3
:1055680063791B041A43A3791B061A436B4BDA6051
:10557800D2E0D378127912021A4363791B041A43D2
:10558800A3791B061A43654B1A61C5E0D3781279D3
:1055980012021A4363791B041A43A3791B061A43A0
:1055A8005E4B5A61B8E01179D378090219435379EF
:1055B80000201B04194393791B0619432EE0117927
:1055C800D37809021943537900201B0419439379AE
:1055D8001B06194330E01179D3780902194353792E
:1055E80001201B04194393791B06194316E011790E
:1055F800D37809021943537901201B04194393797D
:105608001B06194318E01179D37809021943537915
:1056180002201B04194393791B06194304F084FEE6
:105628007AE01179D37809021943537902201B04CF
:10563800194393791B06194304F09BFE6CE0D37859
:10564800127912021A4363791B041A43A3791B06C1
:105658001A43324B9A615FE0D378127912021A43E7
:1056680063791B041A43A3791B061A432B4BDA618F
:1056780052E0D378127912021A4363791B041A4351
:10568800A3791B061A43254B1A6245E0D378127991
:1056980012021A4363791B041A43A3791B061A439F
:1056A8001E4B5A6238E0D378127912021A43637992
:1056B8001B041A43A3791B061A43184B9A622BE062
:1056C800D378127912021A4363791B041A43A37917
:1056D8001B061A43114BDA621EE0D37812791202C4
:1056E8001A4363791B041A43A3791B061A430B4B0D
:1056F8001A6311E0D378127912021A4363791B04F2
:105708001A43A3791B061A43044B5A6304E0032285
:1057180000E00422034B1A7038BDC0462C09002053
:1057280058000020F8030020F0B5061C85B00D1CB9
:10573800141C002949D0002847D0814245D0570180
:10574800FFB206233B43191C0020019304F080FE9E
:105758000C2139430290002004F07AFE0390301C9B
:1057680007F044FD061C281C07F040FD011C301CF6
:1057780007F0C2F9071C029807F038FD391C07F03A
:10578800BBF907F0A1F9051C039807F02FFD391C98
:1057980007F0B2F907F098F9061C002D00D1012591
:1057A800002E00D10126381C094907F065F90028A8
:1057B80003D0201C311C04F0D6FC2A1C00200199BF
:1057C80004F0CAFB034B01221A5505B0F0BDC046D0
:1057D8000000A04158000020F8B50C4D041C2B5CBB
:1057E800002B11D0C6B2730106211943084B87005C
:1057F800FA58C9B2002004F0A1FB064B301CF95836
:1058080004F0B1FC00232B55F8BDC0465800002019
:105818001008002004040020F0B5CF4FCF4C3B788F
:105828006422227063703E79FA78360216437A79D8
:1058380087B012041643BA79C84D1206164366603B
:105848003C1C212B01D101F0F0FA6CD80E2B01D1B0
:1058580000F05FFF2FD8072B00D120E311D8032BCE
:1058680000D154E107D8012B00D1EDE0022B00D183
:1058780020E101F0AFFD052B00D108E300D80FE1CE
:1058880009E30A2B01D100F0AEFD0BD8082B01D19A
:1058980000F03FFC092B01D001F09CFDFFF746FC0E
:1058A80001F09AFD0C2B01D100F0EBFE01D800F0BD
:1058B800CAFE00F0FCFE182B01D101F082F817D8BF
:1058C800142B01D100F0B0FF09D80F2B01D100F043
:1058D8003BFF132B01D100F06AFF01F07BFD162B73
:1058E80001D101F05BF801D800F0C5FF01F05AF8CA
:1058F8001C2B01D101F087F908D81A2B01D101F02E
:105908007FF801D801F06BF801F08BF81F2B01D15B
:1059180001F0D8F901D901F026FA1E2B01D100F0C7
:10592800A4FE01F057FD802B01D101F061FB4AD89C
:10593800402B01D101F04AFB26D8242B01D101F0DC
:10594800C8FA14D8222B01D101F0B7FA232B01D0C1
:1059580001F040FD824B1A78FA705A783A719A78B9
:10596800DB787A71BB71FFF7E1FB01F035FD262B7F
:1059780001D101F0E0FA01D201F0D3FA272B01D1CD
:1059880001F0FBFA01F026FD442B01D101F027FBC1
:105998000AD8422B01D101F01CFB01D901F01CFBF4
:1059A80002F0FAFE01F018FD462B01D101F01DFBB3
:1059B80001D201F017FB472B01D001F00BFD02F0DB
:1059C80014FF01F009FD872B01D101F0B3FB1BD8AF
:1059D800832B01D101F026FB0CD8812B01D101F0DA
:1059E8000BFB822B01D001F0F5FC5E4B02221A76EC
:1059F80001F0F2FC852B01D101F045FB5A4A01D890
:105A080001F030FB01F043FB8C2B01D101F0E7FBE7
:105A18000CD8892B01D101F0B5FB01D201F06BFB49
:105A28008A2B01D101F0C3FB01F0D4FCF22B01D188
:105A380001F070FCFF2B01D101F0C4FC8D2B01D0CB
:105A480001F0C8FC01F0FAFBB97802292ED8454BC1
:105A580001225A54454B00255D54454B281C02220F
:105A68005D5404F02FFBB978062349011943281C1B
:105A7800C9B2404A04F062FAB97808233A79490170
:105A88001943FB7812021A437B79C9B21B041A43E3
:105A9800BB79281C1B061A4304F050FA01F09CFC41
:105AA800BB78022B4ED97A78022A4BD004232B706C
:105AB80001F092FCB9780229F8D82A4B01225A54ED
:105AC8002A4B00255D542A4B281C02225D5404F001
:105AD800F9FAB978062349011943281CC9B2254A9D
:105AE80004F02CFAB97808233A7949011943FB786C
:105AF80012021A437B79C9B21B041A43BB79281CCA
:105B08001B061A43524204F019FA01F065FCB878F2
:105B18000228CBD804F05AF90222B978002004F000
:105B2800D1FAB978082349011943C9B2002004F011
:105B38008BFABB780B4A0121D1540D4A0021D1546C
:105B480001F04AFC6078032800D99CE106F0C8FE01
:105B58001400390069007401DC020020F8030020F9
:105B6800E40300205800002008000020C00800209E
:105B780057080020FF070000181CFFF72DFEA1782A
:105B8800DA4B00255D54DA4B01205D54D94B88402F
:105B98001A78490182431A702279E37812021A436B
:105BA8006379281C1B041A43A379C9B21B061A433C
:105BB80004F0D2F9A178281C2A1C04F083FA01F019
:105BC8000BFC181CFFF708FEA178C84B00265E5492
:105BD800C74B301C5E54022349011943C9B204F073
:105BE80037FC2779E3783F021F436379A1781B04C8
:105BF8001F43A3791B061F43BE4BC7191A78012000
:105C08008840824349011A70C9B2301C3A1C04F01A
:105C1800A3F9A178301C321C04F054FA6F6001F02B
:105C2800DBFB3F221F1C974326D1022B00D93DE7FF
:105C3800142E00DD3AE703225643AF4AF618181C23
:105C4800B600B558FFF7C8FDA178A84B01205F54EE
:105C5800A74B88405F54A74B49011A78C9B28243C1
:105C68001A70381C2A1C04F077F9A178381C3A1CE1
:105C780004F028FA01F0B0FB402F00D09FE0142E6A
:105C880000DD13E700250395049505952A1C191CCA
:105C98001141C80704D502A94A550135032D02D080
:105CA8000132032AF3D10024AC421CDA082212196B
:105CB8006B46D75C381CFFF78FFD7B010221194327
:105CC800C9B2002004F0C4FB03237343DF198A4BD5
:105CD800BF00FB58A200C01AC1174018484003ABC8
:105CE800D0500134E0E7012D37DD039C022D0BD1A4
:105CF80004998C4203DD6B465A7A201C2BE06E46D1
:105D0800081C327A211C26E0049E059DB4420BDD56
:105D1800AC4216DD6846427A311C201CFFF704FDB0
:105D280069468A7A201C0AE0AE420ADD6846027A91
:105D3800211C301CFFF7F8FC69468A7A301C291CA4
:105D480009E06B46211C1A7A281C6C46FFF7ECFC0C
:105D5800627A281C311CFFF7E7FC0024674B0120FE
:105D680099780A1C2241024224D01A79DD7812025D
:105D78002A435D799B792D042A431B061A43032382
:105D88005A435D4B12199200D258584B00255D5466
:105D9800574BA0405D54574BE6B2197881431970B0
:105DA8007101C9B2281C04F0D7F8281C311C2A1C20
:105DB80004F088F90134032CD0D101F00DFB802FB9
:105DC80001D001F009FB142E00DD6FE60025A37851
:105DD80001272B413B422AD02279E37812021A4349
:105DE8006379281C1B041A43A37900261B061A434F
:105DF80003235A43404B52199200D258AF400192A4
:105E0800FFF7EAFCA378394A301CD654384AD654EE
:105E1800384B1A78BA43EFB279011A70C9B2019AAD
:105E280004F09AF8301C391C321C04F04BF9013587
:105E3800032DCCD101F0D0FA5AB2002A01DA01F0D0
:105E4800CBFA032256432C4AF618181CB600B6584B
:105E5800FFF7C2FCA178254B00255D54244B012097
:105E68005D54244B88401A78490182431A70281CD3
:105E7800321CC9B204F070F8A178281C2A1C04F05E
:105E880021F901F0A9FA03232B7001F0A5FAFEF716
:105E980047FB01F0A1FAFEF793FE01F09DFA7B782B
:105EA8009A1F012A09D98C2B07D0C02B05D0C72BE4
:105EB80003D03A32D2B2322A03D8A278002A04D0C8
:105EC800F4E5BA78022A00D9F0E5952B33D8932B5C
:105ED80000D3A5E00D2B19D80C2B00D3A0E0052B7F
:105EE80000D179E00CD8042B70D00EE157080020BF
:105EF800C008002031080020E8020020DC02002051
:105F0800062B6FD0072B00D17BE0FEE0862B63D0F9
:105F180005D8822B00D189E0832B57D0F5E08C2B54
:105F280000D189E08D2B00D0EFE0A0781A2104F091
:105F3800C7F901F051FAC32B00D1ADE016D8B52B43
:105F480000D184E00AD86733DBB2012B00D9DCE04A
:105F5800A078182104F0B4F901F03EFAC12B00D161
:105F680084E000D98DE0C02B4BD0CEE0D22B00D1FD
:105F78009EE013D8C72B35D0CC2B00D0C5E0A37832
:105F8800D74A580111180E3180180233081A5B01DC
:105F9800C018022201F0DEFF01F01EFAD62B00D154
:105FA80095E0FE2B00D1A1E0D42B00D0ADE0A37882
:105FB800CB4A58011118143180180233081A5B01B2
:105FC800C018042201F0C6FF01F006FAA0780621E5
:105FD80004F076F901F000FAA0780C2104F070F9C9
:105FE80001F0FAF9A278BE4B510158180930CB18C4
:105FF8000232C01A52018018597A01F03FFF01F0AD
:10600800EBF9A278B64B510158180A30CB18023276
:10601800C01A52018018997A01F030FF01F0DCF9BA
:10602800A078142104F04CF901F0D6F9A0780421E5
:1060380004F046F901F0D0F9A378002B00D035E53B
:106048004B20A849012201F085FF01F0C5F9A3788A
:10605800A3495A01101C1830023341185B01801AF9
:10606800C018042201F076FF01F0B6F9A0789C4B25
:106078004201D318101C4830197A01F0FFFE01F0D4
:10608800ABF9A178964B881C49014001C918042234
:1060980001F060FF01F0A0F9A078914B4101C91807
:1060A800400104314430042201F054FF01F094F916
:1060B800A3788B495A01101C1030023341185B0138
:1060C800801AC018042201F045FF01F085F9A37871
:1060D800834A580111181C3180180233081A5B01D1
:1060E800C018022201F036FF01F076F9A3787C4A45
:1060F800580111180C3180180233081A5B01C018B6
:10610800012201F027FF01F067F903232B7001F04A
:1061180063F97B789A1F012A09D98C2B07D0C02BE9
:1061280005D0C72B03D03A32D2B2322A03D8A2788C
:10613800002A04D0BAE4BA78022A00D9B6E4952B2A
:106148002AD8932B00D3BEE00D2B10D80C2B00D3EC
:10615800B9E0052B00D17FE002D8042B67D03EE1DF
:10616800062B00D191E0072B00D19DE037E1862B6B
:1061780072D005D8822B00D1ABE0832B57D02EE10B
:106188008C2B00D1B6E08D2B00D028E1A0781A2105
:1061980004F076F801F020F9C32B00D1E6E016D818
:1061A800B52B00D1BDE00AD86733DBB2012B00D98B
:1061B80015E1A078182104F063F801F00DF9C12B5E
:1061C80000D1BDE000D9C6E0C02B6DD007E1D22BCD
:1061D80000D1D7E013D8C72B57D0CC2B00D0FEE086
:1061E800A3783F4A580111180E3180180233081A53
:1061F8005B01C018022201F040FF01F0EDF8D62B38
:1062080000D1CEE0FE2B00D1DAE0D42B00D0E6E0BE
:10621800A378334A58011118143180180233081A28
:106228005B01C018042201F028FF01F0D5F8A0781E
:10623800062104F025F8A57806216B011943C9B297
:10624800002003F02BFF284BAD00E850A378274A25
:106258000021D15401F0C0F8A0780C2104F010F806
:10626800A5780C216B011943C9B2002003F016FF71
:106278001F4BAD00E850A0781C4A00211154820041
:10628800D15803F070FF01F0A7F8A378144A5C0115
:1062980010190930A41802335B01001BC01801F063
:1062A800D4FE607201F098F8A3780D4A5C011019C9
:1062B8000A30A41802335B01001BC01801F0C5FEA8
:1062C800A07201F089F8A078142103F0D9FF01F039
:1062D80083F8A078042103F0D3FF01F07DF8C046CD
:1062E800C8080020D308002010080020580000200B
:1062F80004040020A378002B01D0FFF7D7FBA049A6
:106308004B2001220D1C01F0B8FEA0780B3D430183
:10631800ED18EB7A0821C91AC9B202F025FC01F080
:106328005BF8A37897495A01101C183002334118BA
:106338005B01801AC018042201F09FFE01F04CF89E
:10634800A078904B440140014830E41801F07DFEEC
:10635800207201F041F8A1788A4B881C490140015C
:10636800C918042201F089FE01F036F8A078854B9F
:106378004101C918400104314430042201F07DFE76
:1063880001F02AF8A3787F495A01101C1030023313
:1063980041185B01801AC018042201F06EFE01F05A
:1063A8001BF8A378774A580111181C31801802335A
:1063B800081A5B01C018022201F05FFE01F00CF818
:1063C800A378704A580111180C3180180233081A42
:1063D8005B01C018012201F050FE00F0FDFF03230D
:1063E8002B7000F0F9FFBB78022B00D198E0032B4B
:1063F80000D19BE0002B00D00CE17B78502B62D0C1
:1064080024D8462B50D00FD8422B46D006D8402B44
:106418003FD0412B00D0FBE05B4B7AE05A4A442B3B
:106428003ED03FD81379F1E04C2B45D008D8492B02
:106438003CD04B2B3DD0472B00D0E9E0524B99E0A4
:10644800514A4E2B3BD03CD8537DDFE0812B4BD0BB
:1064580011D8542B3ED005D84B4A522B36D037D8BA
:10646800137DD3E0562B3BD037D3802B00D0CFE021
:10647800464B1B7ECAE0852B40D004D8832B39D0ED
:106488003AD8424BAFE0FE2B42D044D8F02B3FD055
:10649800BEE03F4801F0D9FD93E03B4B5B78B5E0A7
:1064A800D26941E05379B1E0374B66E0364BDB7D8A
:1064B80033E0354BDB78A9E0334B9B78A6E0D38CEF
:1064C800A4E0537EA2E0304B9B7D9FE0126A2BE054
:1064D800126929E02C4B9B7E98E02B4BDB7E95E0E4
:1064E800294B0533DB7F91E0284B1B7E043B5A4246
:1064F80053418BE0254B3AE0264B35E0234A264BA7
:106508009668264873431B1893605B005B087DE020
:10651800234B1B787AE0234B1B785A1E934175E076
:106528007A78214B9200D2586A6075E078782E28E4
:106538006ED806F0CBF9181B1E6D6D6D6D6D6D2153
:106548003D406D6D6D6D6D6D6D6D6D6D6D6D6D6DD0
:106558006D43484A4C4E506D6D6D6D6D6D54575A74
:106568005D6063666900114B1B684FE00F4B5B6809
:106578004CE00E4B9B6849E00C4BDB6846E0C0469C
:10658800D3080020C8080020080000205800002078
:10659800FF070000F40300206D4EC64139300000AB
:1065A80069090020F2030020100400202C090020B3
:1065B800C14B1B692AE0C04B5B6927E0002003F050
:1065C800FFFE686028E0002006E00120F7E70120D0
:1065D80002E00220F3E7022003F004FFF1E7B64BE4
:1065E8009B6913E0B44BDB6910E0B34B1B6A0DE009
:1065F800B14B5B6A0AE0B04B9B6A07E0AE4BDB6AC3
:1066080004E0AD4B1B6B01E0AB4B5B6B6B6003E0D5
:10661800032300E004232B70A84B1B78002B01D127
:1066280000F0DAFEA64B696808221960A54B00291C
:1066380004D119680A431A6000F0CEFE1C6894431E
:106648001C6000F0C9FEBB78022B16D17978372977
:106658000FD8A72676009C4B881989008000C91896
:10666800042201F077FC00F0B7FE7B78142B00D8E9
:10667800CDE203232B7000F0AFFE04232B7000F053
:10668800ABFEBB78022B0ED179783729F1D8A72237
:1066980052008D4B881889008000C918042201F027
:1066A800ECFC00F099FE04232B7000F095FEB878FE
:1066B800022801D9FFF7FAF97B78012B08D0002BC3
:1066C80002D0022B08D020E003F076FB00F084FE15
:1066D80003F07CFB00F080FE03F082FB774B6860E0
:1066E8001B78002B01D100F077FE754B082218604B
:1066F800744B002804D11C6822431A6000F06CFE19
:106708001E6896431E6000F067FE03232B7000F09E
:1067180063FEBB78002B02D0022B05D00FE0301CA3
:10672800FDF718FE00F058FE7878002E03D1FDF72B
:1067380065FD00F051FEFDF73FFD00F04DFE634C96
:106748000423237000F048FEBB78012B11D0002BE6
:1067580005D0022B12D17878FDF7A4FD0CE07878EB
:10676800082802D8FDF76CFD06E00A2808D16B60FE
:1067780006E0787803F0A2FF686001E004232B703C
:106788004E4B1B78002B01D100F026FE4C4B69685C
:10679800082219604B4B002904D11E6832431A6045
:1067A80000F01AFE18689043186000F015FE78781B
:1067B800434C092829D806F089F805080B0E141A45
:1067C8001D20232721688E191EE02268961B1BE0D6
:1067D80023685E4318E02068311C06F0D9F8206071
:1067E80013E02068311C06F029F921600DE02068CB
:1067F800064009E021680E4306E02268564003E09F
:106808002668F343236000E02660216808222D4BA8
:10681800002904D1186802431A6000F0DDFD1968E8
:106828009143196000F0D8FD254B1A68254BB242F8
:1068380005DD1C6803218C43211C04200CE0B242B6
:1068480005D11E6806218E43311C012004E018681A
:1068580005218843011C0220014319600821002AF0
:1068680004D11A681143196000F0B6FD1A688A430A
:106878001A6000F0B1FD78780C2801D900F0ACFD61
:10688800104B06F023F80710273039424C555E6745
:10689800707982001B681C0701D400F09DFD0C4B29
:1068A800DE6100F099FD1B68180701D500F094FD22
:1068B800074BDE6100F090FD2C090020F303002057
:1068C800E4030020E402002010040020F803002064
:1068D800580000201B68D90701D400F07DFDDB4B70
:1068E800DE6100F079FD1B68DA0701D500F074FD60
:1068F800D64BDE6100F070FD1B685C0701D400F028
:106908006BFDD24BDE6100F067FD1A6805231A4261
:1069180001D100F061FDCD4BDE6100F05DFD1B682B
:10692800980701D400F058FDC84BDE6100F054FD13
:106938001B68990701D100F04FFDC44BDE6100F0E0
:106948004BFD1B68DA0601D400F046FDBF4BDE6143
:1069580000F042FD1B689C0601D400F03DFDBB4BD6
:10696800DE6100F039FD1B68580601D400F034FDE3
:10697800B64BDE6100F030FD1B68190601D400F04B
:106988002BFDB24BDE6100F027FD1B68DA0501D450
:1069980000F022FDAD4BDE6100F01EFDAB4BDE6169
:1069A80000F01AFDA94B1A6A072A01D900F014FD54
:1069B800511CDC6992009A1819625462DE6100F079
:1069C8000BFDA24B1A6A002A01D100F005FD013A1D
:1069D8001A6292009A18526ADA6100F0FDFC7B781C
:1069E8002E2B04D89A4A0121D15400F0F5FCFF2B34
:1069F80000D03EE6954B012244331A7000F0ECFCBF
:106A08007B782E2B04D8924A0021D15400F0E4FC64
:106A1800FF2B00D02DE68D4B002244331A7000F076
:106A2800DBFC8A4D2B1C45331B78002B10D10A2325
:106A3800701C04D1874A16687343AB6401E05E4357
:106A4800AE6401F061FE2B1C45330122E8641A7024
:106A58006078042801D900F0BFFC05F037FF034136
:106A680070A3170001F050FEE96CAB6C401AC21716
:106A780080185040984204D9453500232B7000F007
:106A8800ABFCEB69013BEB6100F0A6FCA07803F0DE
:106A9800A7F9002808D1704B10221C68453594438B
:106AA80028701C6000F098FCAE6C002E13D001F02A
:106AB8002BFEE96CAB6C401AC21780185040984204
:106AC80009D9002345352B70634B10221C682243DB
:106AD8001A6000F081FCEB69013BEB6100F07CFC83
:106AE800002003F0C2FAA478012364002041041CAA
:106AF8001C4009D0002345352B70574B10221E68C7
:106B080096431E6000F068FCA86C002812D001F0C3
:106B1800FBFDE96CAB6C401AC217801850409842D4
:106B280008D94D4B45352C701C68102222431A6039
:106B380000F052FCEB69013BEB6100F04DFC03AE49
:106B480000207C21321C03F097FAA4780223640009
:106B5800A3401C1CB3781C4009D0002345352B707A
:106B68003D4B10221E6896431E6000F035FCA86C51
:106B7800002812D001F0C8FDE96CAB6C401AC217AE
:106B880080185040984208D9334B45352C701C6802
:106B9800102222431A6000F01FFCEB69013BEB61F5
:106BA80000F01AFC03AE00207C21321C03F064FACA
:106BB800A478B378640023411C1C01231C4009D02D
:106BC800002345352B70244B10221E6896431E6007
:106BD80000F002FCA86C002811D001F095FDE96CCA
:106BE800AB6C401AC21780185040984207D91A4B0C
:106BF80045352C701C68102222431A60ECE3EB69BF
:106C0800013BEB61E8E3114B00221A76E4E3BA7822
:106C1800022A27D803245C431049A418A40010486A
:106C28006650807E002800D1D6E3002B00D1D3E344
:106C3800013B0C205843C326F600801992008018A7
:106C48006118042201F086F9C6E3C0465800002006
:106C58007E090020E4030020E4020020E80200206E
:106C680008000020FF2A01D0FEF720FFCC4E002BA1
:106C780012D103239C00271CDD1C0C37C9490422B0
:106C880060183119043401F065F9BC42F6D13F2D82
:106C980000D1A1E32B1CEDE70025637803215A1EE0
:106CA80059430C205043C322D20069188018890028
:106CB800AA00801871180422013501F04BF9032D40
:106CC800EBD189E37B78142B00D9D2E4BA78022A75
:106CD80019D803214B43B2499A18B34B9200525822
:106CE8001B786A60002B00D176E3B04B08211A604C
:106CF800AF4B002A03D11C68214319606CE31A6862
:106D08008A431A6068E3FF2A01D0FEF7CFFEA44E3B
:106D1800002B12D103239C00271CDD1C0C37A14932
:106D2800042260183119043401F0A7F9BC42F6D1E5
:106D38003F2D00D150E32B1CEDE70025637803219C
:106D48005A1E59430C205043C322D2006918801898
:106D58008900AA00801871180422013501F08DF904
:106D6800032DEBD138E37F78142F00D981E4A6787E
:106D780073B2002B2EDA0025A3782B41DE070DD540
:106D88006B0102211943C9B20020667803F060FB49
:106D980003235E43824B7619B600F050854B9B7EE9
:106DA800002B13D06378002B10D05A1E0C205043B0
:106DB800C321C900401803215943AA008018691843
:106DC800774A89008918042201F0C4F80135032D97
:106DD800D2D101E3022E01D9FEF768FE7301022128
:106DE8001943C9B2002003F033FB03256F436C4AF3
:106DF800BE19B6006F4BB0509B7E002B00D1EBE262
:106E08006378002B00D1E7E2A178581E0C24604378
:106E18006B43C324E40000198C00C9188900891841
:106E28000019042201F096F8D6E278785F4C0A2817
:106E380036D8614B05F04AFD060A0F13191F2327A0
:106E48002B2E30001B682668F31802E01B682068A8
:106E5800C31A236024E01B6821684B43F9E72068C4
:106E6800196805F095FD20601AE02068196805F09A
:106E7800E5FD216014E01B6822681340E9E71B6800
:106E880026683343E5E71B6820684340E1E7196853
:106E9800CA4304E0226802E01E68226826601A607D
:106EA80021680822424B002903D1186802431A605E
:106EB80092E21968914319608EE23C4B1A78FA7095
:106EC8005A783A719A78DB787A71BB71FDF728FBAA
:106ED80082E27878052800D97EE2354B05F0F6FC89
:106EE80003080D12171C1C680F2222401A6073E257
:106EF8001E68102296431E606EE218682022904396
:106F0800186069E2196840229143196064E21C68BC
:106F1800802294431C605FE21E68284A32401A604F
:106F28005AE27B782E2B01D9FFF7A3FB244A9B005A
:106F3800D3181E6550E2234B1C4AD86819691060A3
:106F48001D4A9E6911601E4A19495C690E60D8691C
:106F5800111C45310870D461196A5C6AD164946463
:106F68001A1C283212781849885C002801D00120A0
:106F780088542C3300221A702EE2BB78022B01D9D8
:106F8800FEF794FD7A78142A01D9FFF772FB0321E2
:106F98004A43D318054A024912689B005A501BE21B
:106FA800E80200200C060000F3030020E4030020A0
:106FB800E40200200800002000040020FFFEFFFF7C
:106FC80058000020580100207E09002001F0BAFB7B
:106FD80002E201F005FCFFE101F003FCFCE101F035
:106FE80001FCF9E101F0FFFBF6E101F0FDFBF3E143
:106FF800B34B00221A76EFE17B78002B02D0012BED
:1070080004D00CE0AE4B01221A76E5E1AD4A964277
:1070180001D9FEF74BFDAA4A1376D661DCE10323BA
:107028002B70D9E1A64A0021131C44331970A64BD2
:107038002C331970131C0124880050336442C45047
:10704800A2480023435401312F29F3D11376D36189
:107058001362453213709E4A13609E4A13609E4A1B
:107068001360B9E1137D98070AD4964B9E4201D963
:10707800FEF71CFD924B04221A76934B1E63ABE17C
:1070880008232B70A8E18E4B00221A76A4E1934BBB
:1070980001271F709378924C23708A4B9E4220D808
:1070A800137D3B4001931CD103AD301C291C00F01B
:1070B800FDFD2B78019E63706B78A370AB78E3704D
:1070C800AB7923716B7963712B79A371EB78267295
:1070D800E371E25D237A0137D3182372082FF8D1C0
:1070E8007AE10123E218002101331170082BF9D14C
:1070F8002378237270E17B78002B10D1774A012125
:1071080011707849764A897811707749086801338F
:10711800C11801390978D154082BF8D15CE1012B49
:1071280000D059E10422EA716B7156220823AA7132
:107138002B7151E17878032800D94DE105F0C6FBA1
:10714800020E1A1E5E4B1A7E45331B78EA71AB712C
:107158005D4B1B6B1A0A6A712B713DE1584B1A7E05
:10716800EA711A1C45321278DB69AA711A0A6A7127
:107178002B7131E1564B1B686B602DE1554B1B6839
:107188006B6029E17B78002B00D025E1B9780029D4
:1071980000D021E1554B9E4200D01DE1494800F046
:1071A8006DFE00F0C5FD0120FDF704F914E17A78C1
:1071B8004F4B002A00D001221A70E2784D4B1A700A
:1071C800414B343319784C4B19704C4900230B70E0
:1071D8004B490B704B4B19780A431A70FCE07C78CA
:1071E800002C02D0012C19D024E04748042203A91E
:1071F80000F043FF3B79FA781B0213437A7903982E
:1072080012041343BA7912061343834203D13F4C45
:1072180001236360E0E03D4E7460DDE0BB782A2B1B
:1072280005D139483A49042200F094FED4E00323FA
:107238002B70D1E0354C03232370CDE078780328F8
:107248003AD805F043FB06022B361F480023816B12
:107258000DE01D4B9A6B092A05D8511C92009963C1
:107268009B18DE63B8E009232B70B5E001338B422D
:1072780000D1B1E0051C3C359A005459B442F5D10F
:10728800AD1800224C1E0432A34205D2AC18AE58E9
:10729800043C01332660F5E784639DE00A4A002335
:1072A8009363111C3C31002058500433282BF8D12B
:1072B80092E00A236B608FE003232B708CE0C046BA
:1072C80058000020FF070000580100207E09002018
:1072D800E403002000040020E4020020E80300206A
:1072E800E90300200800002004000020D204000068
:1072F800300800205B080020740900205A0800208C
:10730800AD09002031080020FB070000F803002029
:10731800DF0200207B78812B5ED1BB78922B5BD17A
:10732800BB79A32B58D17B79B42B55D13B79C52B8D
:1073380052D1FB78D62B4FD1284B8022D203DA6268
:10734800274B34331B78072B2AD101F0DDF9051CB4
:1073580001F0DAF9401BC117224C40184840A042FE
:10736800F6DD03F045FD204A8023DB04D3671F497F
:10737800C02252008B50F0220121920230231C4877
:1073880004F082FE01F0C0F9051C01F0BDF9401BB4
:10739800C21780185040A042F7DD0120FDF70AF817
:1073A800FDF706F8002004F045FC05F02BFA002153
:1073B8000A1C032005F0FAF905F03EF80D4B0122EE
:1073C8001A7009E00C4B9E4206D1054B012264332A
:1073D8001A7001E002232B7007B0F0BD00100540C1
:1073E80058010020E703000004E100E000E100E0AC
:1073F8000000014068090020D2040000F7B5344AB3
:1074080000231360334A344E1360344AF361136027
:10741800321C453213701C1C6701FFB20621394328
:10742800002003F015F82E4BA5000C2158513943C4
:10743800002003F00DF82B4B01345851032CEBD1ED
:10744800294B0821DB7A0020C91AC9B201F08CFB4C
:107458000023264A00209918802204330860D200AD
:107468009342F6D1224D0327AB7E834211D0BC0054
:10747800221C0C32033701921E4A1F49A018091911
:10748800042200F0FAFD019B04349C42F4D13F2F02
:10749800EDD1EB7E002B09D06B1DD97F002002F0C7
:1074A80049FE6B7D002B11D001230FE0A724E400D7
:1074B8000E4B124A201C99180919042200F0DDFD10
:1074C8000434C323DB009C42F2D1E5E73376F7BDF1
:1074D800E40300200004002058000020E4020020FB
:1074E8001008002004040020C80800201004002010
:1074F800080000200C060000E8020020C8FAFFFF80
:10750800F0B5104C85B002AE0192351C271C8C4694
:1075180006CF06C50C4D019AEB70AA701A0A2A719B
:107528001A0C1B0EAB71094B61466A710022287058
:1075380069701A70FEF770F9606806CE06C405B067
:10754800F0BDC046F8030020DC020020F303002051
:10755800F7B51D4F6B463A1C0C1C42CA42C31B4B65
:10756800427800261A7082786D465A70C2789A70EE
:1075780002799A7142795A7182791A71C279DA70EC
:10758800134B1E70FEF748F9124B1A783B1CB24297
:107598000ED1227062703A78A2707A78E270FA7925
:1075A8002271BA7962717A79A2713A79E27108E046
:1075B800012A06D1084AB2185278A2550136082E77
:1075C800F8D103CD03C3F7BDF8030020DC02002087
:1075D800F3030020E8030020E9030020F0B5D24BB4
:1075E80091B01B78D14D002B0DD0D14B1B78062BB9
:1075F80009D00A2B07D0102293430F2B03D02B1C42
:10760800343300221A702B1C34331A78531ED9B223
:10761800012931D8C74908A8CA6842605A1E93414F
:10762800073303702B1C6533C34A1B7812784370E9
:10763800002383709A4210D18B680372BF4B19786C
:10764800417259788172D979C172997901735979DE
:1076580041731B79C273837308E0012A06D1B849C4
:107668000133C95CC218D171082BF8D100F01CFF96
:10767800002800D1FDE2ACE0032A21D1AE4B1B78F3
:10768800002B11D1AB4EAD4CB07877782378C71961
:10769800FF186378FF18E379FF18A379FF18637957
:1076A800FF182379FF1818E0012B00D091E000247F
:1076B800A34B185D013400F023FE092CF8D188E0B3
:1076C8000023042A25D19D4C01229A4E6370227012
:1076D8006360B0787778C719BF1800F011FE70782A
:1076E80000F00EFE207800F00BFE607800F008FE37
:1076F800E07900F005FEA07900F002FE607900F064
:10770800FFFDFFB2207900F0FBFD381C00F0F8FD0A
:107718005FE0072A3FD1884A1278002A25D1854B95
:107728009F785B789C46854B5A795C78D8799979AB
:1077380001921E781B79624600936B465A72019A31
:107748001F7267449E729A73F619009ADC72A41924
:1077580018735973DA730019019B0918009C5A1899
:10776800A3186F463B7400240BE0012AFBD1744A2E
:107778000820D25CC018694601334254092BF6D15F
:10778800F1E7082212196B46D05C013404F0F2F8D4
:10779800092CF6D11DE0082A1BD1684A0120537034
:1077A80010705360634A6C46917852782172627205
:1077B8008A181218A072E37223736373A373E373B6
:1077C80022741C1C02AF385D013404F0D3F8092C74
:1077D800F8D15C4B1A78002A63D05B4B5B4E187863
:1077E8000138062859D805F071F804041B58585870
:1077F8003E00504A0CA89168802301723178D26803
:1078080043728A238372817300230721C37203732F
:107818004373017043708370426000F045FE3CE0A2
:10782800444C3378A0786778C7190A37FF1800F0F6
:1078380067FD607800F064FD802000F061FD8A201B
:1078480000F05EFD002000F05BFD002000F058FD18
:10785800002000F055FDFFB2307800F051FD381CD3
:1078680000F04EFD19E0334B05AC99785A7833781F
:1078780062708A1880200A320027A070E3718A207B
:107888009B182170E07027716771A7712372E05D02
:10789800013704F06FF8092FF9D12A4C002333700F
:1078A8002370224C0023221C34321370224A137096
:1078B800231C64331B78002B02D00120FCF77AFDCF
:1078C80008AE301C00F02CFE071E49D0327A184B47
:1078D8001A70727A5A70B27A9A70F27A9A71327B06
:1078E8005A71727B1A71B27BDA707278231C653315
:1078F8001A7000F009FF164B00221860154B1A7019
:107908003278231C3433072A01D1012200E00222F5
:107918001A70114B1A7E114B511E012902D9052AE2
:1079280000D0A9E00022C4E0F203002058010020A2
:10793800DC02002008000020E8030020F8030020F3
:10794800E9030020AD090020740900205A0800202E
:10795800640900202008002058000020F3030020BC
:1079680005A800F0E7FC061E53D000F0FFFC002835
:1079780002D0231C66331F70231C663318786F46A9
:10798800421C211C3E7DD2B267311A700E54092A5E
:1079980000D091E000221A70B74B09785B789942C1
:1079A80000D089E0111C231C6733D05C0132091810
:1079B800C9B2082AF7D11A7A261C34368A4225D148
:1079C8005978AE4A117099785170D97891701979AF
:1079D80091715979517199791171DB79D37000F0EE
:1079E80093FEA74BA74A1860002313700322327036
:1079F800221C66321370A44A117EA44A481E01282C
:107A080002D9052900D00123137055E004233370EF
:107A180052E00CAF381C03F0BFF9002834D0331CF7
:107A2800BA5D01369B18DBB2082EF9D13A7A9A4230
:107A380026D1924B7A781A70BA785A70FA789A7076
:107A48003A799A717A795A71BA791A71FA79DA7037
:107A580000F05AFE8A4B8B4A186000231370221CD0
:107A6800343207211170884A191C127E874B501E28
:107A7800012803D9052A01D001221AE019701BE058
:107A8800231C34331E7017E07F4B1A7E013A012AFB
:107A980012D8DA697E498A420DD8511CD961101C66
:107AA800764900F003F9231C343309221A70774B06
:107AB80001221A7000E01876734B187E1E1C0428E9
:107AC80005D16E4F39784AB2002A00DBA2E0231CA8
:107AD80034331B780422181C904305D0082B03D09C
:107AE800062B01D0FDF798FE231C34331B78092B95
:107AF8006FD100F009FEF168664F401AC2173B6863
:107B080080185040984208D9634B1A78012A01D14D
:107B180002221A7000F0F8FDF06000F0F5FD3169FE
:107B28007B68401AC21780185040984208D95A4BAF
:107B38005A78012A01D102225A7000F0E5FD30611D
:107B480000F0E2FDBB687769C01BC11740184840C8
:107B5800984208D9504B9A78012A01D102229A708A
:107B680000F0D2FD7061331C44331B78002B30D0F9
:107B7800231C2C331B78002B2BD1474AD15C0229BC
:107B880024D1311C5031980041584F1C1CD0434A15
:107B9800F06912686861EA60414AF76C12682F62FE
:107BA8002A61404AF1611268AA61321C4532107894
:107BB800E861B06C6862281C2830037000231370D9
:107BC8002C3501232B7004E00021D15401332F2BD5
:107BD800D3D1231C34331B78092B04D1327E022ADB
:107BE80001D105223276A26B002A42D0092B40D15E
:107BF800337E012B3DD1F1690023201C3C309D00D0
:107C08002858814202D10523337632E0013393426A
:107C1800F3D12EE0221C34321278151C854328D06B
:107C2800082A26D0062A24D01F4D206B69703A797D
:107C3800F97812020A43797909040A43B9790906DD
:107C48000A436A60124A90420FD8391C00F04DF975
:107C5800206B391C00F0B0F80723002803D0236BF1
:107C68000133236365232B7003E007222A70002267
:107C78001A7611B0F0BDC04608000020DC020020D2
:107C88006C0900207309002058000020F30300202D
:107C9800FF0700002C0900207E090020E4030020D3
:107CA80000040020E4020020F803002038B507256E
:107CB800454380231B01ED180C1C002203210220E0
:107CC800FCF7F8FB290AC9B200220220FCF7F2FBF4
:107CD800E9B200220220FCF7EDFB00210A1C022079
:107CE800FCF7E8FB002120700A1C0220FCF7E2FBED
:107CF800002160700A1C0220FCF7DCFB0021A07048
:107D08000A1C0220FCF7D6FB0021E0700A1C0220A6
:107D1800FCF7D0FB002120710A1C0220FCF7CAFBEB
:107D28000021607101220220FCF7C4FBA07138BD5C
:107D380038B580242401022006210122FCF7BAFB71
:107D4800052100220220FCF7B5FB022000210122B8
:107D5800FCF7B0FB02252842F2D0291C281C00227F
:107D6800FCF7A8FB210AC9B2281C0022FCF7A2FBD9
:107D7800281CE1B20022FCF79DFB00252A1C3F3A93
:107D880053425A41D2B2022000210135FCF792FB3E
:107D9800402DF3D1052100220220FCF78BFB0220A5
:107DA80000210122FCF786FBC307F3D4802340346B
:107DB800DB019C42BFD138BDF7B507254543802379
:107DC8001B01ED180C1C002203210220FCF772FB9A
:107DD800290AC9B200220220FCF76CFBE9B2002292
:107DE8000220FCF767FB00210A1C0220FCF762FB5B
:107DF80000210A1C071C0220FCF75CFB00210A1C5E
:107E0800061C0220FCF756FB00210A1C051C022058
:107E1800FCF750FB6B460021D8700A1C0220FCF7C7
:107E280049FB6B46002118710A1C0220FCF742FB33
:107E38006B465871002102200122FCF73BFB6B4680
:107E4800987123780020BB4217D16378B34214D1CC
:107E5800A378AB4211D16B46DA78019B20791B02DB
:107E68001343E27800021043627912041043A279A6
:107E780012061043181A43425841FEBD70B501223C
:107E8800051C0E1C02200621FCF714FB052100220C
:107E98000220FCF70FFB022000210122FCF70AFB5D
:107EA80002242042F2D0211C0022201CFCF702FBF5
:107EB800290AC9B20022201CFCF7FCFAE9B2002208
:107EC800201CFCF7F7FA201C311C0122FCF7F2FAFF
:107ED800052100220220FCF7EDFA022000210122F0
:107EE800FCF7E8FAC307F3D470BD38B50725454356
:107EF80080231B010C1CE8180978FFF7BFFF0F4B04
:107F08006178E818FFF7BAFF0D4BA178E818FFF77A
:107F1800B5FF0C4BE178E818FFF7B0FF0A4B217961
:107F2800E818FFF7ABFF094B6179E818FFF7A6FFE0
:107F3800074BA179E818FFF7A1FF38BD0108000039
:107F480002080000030800000408000005080000FB
:107F580006080000F7B5041C0191171C0220062131
:107F68000122FCF7A7FA052100220220FCF7A2FA59
:107F7800022000210122FCF79DFA02252842F2D0B6
:107F8800291C281C0022FCF795FA210AC9B2281CD2
:107F98000022FCF78FFA281CE1B20022FCF78AFACB
:107FA8000025BD4244D0019B01343F26595D26403F
:107FB8000122002E03D07A1EAA1A53425A41D2B285
:107FC8000220FCF777FA002E30D17B1E9D422DD27D
:107FD800052100220220FCF76DFA0122022000216F
:107FE800FCF768FA01221042F2D102200621FCF7C0
:107FF80061FA052100220220FCF75CFA0220002128
:108008000122FCF757FA02263042F2D0311C002236
:10801800301CFCF74FFA210AC9B20022301CFCF7C9
:1080280049FAE1B2301C0022FCF744FA0135B8E7FE
:10803800052100220220FCF73DFA0220002101223E
:10804800FCF738FAC307F3D4F7BD10B50321041CB5
:1080580000220220FCF72EFA210AC9B200220220CF
:10806800FCF728FAE1B200220220FCF723FA0021EB
:1080780001220220FCF71EFA10BD70B5041C0E1C6C
:10808800151C032100220220FCF714FA210AC9B2A8
:1080980000220220FCF70EFAE1B202200022FCF7CF
:1080A80009FA0024AC420BD06A1EA21A53425A4164
:1080B800D2B202200021FCF7FDF930550134F1E776
:1080C80070BD37B5052100220220FCF7F3F9022024
:1080D80000210122FCF7EEF97123041C1C40F1D1A8
:1080E80000F012FB051C00F00FFB401BC317C01863
:1080F8005840344B984209DC002C09D13248FFF72C
:10810800A4FF041CAA3C63425C41ECE7002C03D0AA
:108118002E4B1B78002B3CD02B480021FFF7AEFEDE
:10812800FFF706FE00202A494022FFF713FF00242C
:10813800B422101C60430130FF302649FFF70AFFC4
:10814800A01C4001244920220134FFF703FF032C1F
:10815800EED10023C3240193E400201C01A90422CA
:10816800FFF7F8FE0434FF23DB009C42F5D100231F
:10817800A7240193E400201C01A90422FFF7EAFECA
:108188000434C323DB009C42F5D10F48AA21FFF732
:1081980075FE00200E494022FFF76FFF0F4C40206C
:1081A800211C2022FFF769FF211C2031602020229A
:1081B800FFF763FF211C403180202022FFF75DFF7D
:1081C80037BDC046CF070000FF0700006808002041
:1081D8000800002020E3000000E30000C808002099
:1081E800254A30B5506A53691840C1071CD5234B3E
:1081F8005B6B990601D5936A16E0214B1C68611CDC
:108208001F3C651EAC41644221405C68A14205D018
:108218001C68956A1C19EDB2257219601949052464
:108228000C60996A184B1960830723D5164B196897
:1082380000291FD1124BDC6A186B844211D00F48F9
:108248002024C46203205061186B441C1C631C1C4E
:108258003434205CC0B2D0621A6B202A0AD1196368
:1082680008E0536A990505D5034B01225A61034B6F
:1082780020221A6330BDC046001008400010054097
:10828800C8010020B4090020B009002037B5184BF8
:10829800051C01200024021C04215C601C601C6376
:1082A8001C6004F03FF80120021C032104F03AF896
:1082B8000120032104F070F80E4B0F49AD00202275
:1082C8001A6369580D4B01225A609A6019638C2110
:1082D800090119615021D96001A85A610F2303705F
:1082E800032343708470C27004F0EAF837BDC046B7
:1082F800C80100200010054050E3000000100840AD
:108308000A4B10B5D96A4A1C1F394C1EA141494273
:108318000A40196B8A4207D0D96A1C1C343460544D
:10832800DA62034B03225A6110BDC046C80100201F
:1083380000100840094B59681A6891420CD05A68D5
:10834800511C59609A18127A02705A680120202A22
:1083580003D100225A6000E000207047C8010020C5
:10836800014B98627047C046C8010020034B0020AB
:108378001A78824201D0187001207047B80900208D
:10838800F8B5071C0E1C00201321151C012203F050
:10839800C9FF00200122142103F0C4FF314B02223F
:1083A8001A6504221A6601221A6608221A662E4CD9
:1083B8002E4A781E2265072815D804F087FA12106D
:1083C8000E0C0A1408042A4A5A66012213E0294AA4
:1083D800FAE7294AF8E7294AF6E7294AF4E7294A51
:1083E800F2E7294AF0E7294AEEE7196F8802FCD438
:1083F8000132212A06D000212163616324491143F7
:108408006162F2E7710580273F062248C9083943AF
:108418002063BC466163204F84214901A163B603F0
:108428006762C027B60B3F063E43206366631B4E58
:10843800A1630D4A6662002D10D06C05E4086646FB
:108448003443AD031063AD0B5463154C2F43916354
:1084580054621063576391631249516212221A667B
:10846800F8BDC04600000E40FC000E400000750C30
:1084780001706B0003707A000F707A000F707F0034
:108488001F707F004F707F009F707F0007707A0019
:10849800809F0000FFFFFFDF829F0000839F000096
:1084A800849F0000859F000010B5C27A837A120667
:1084B8001B041A43037A1A43437A1B021A43144BC8
:1084C8009A60C17B827B090612040A43017B0A4336
:1084D800417B09020A43DA60447841680D4A002C5E
:1084E80003D089038C0BE02102E04905CC08A021C8
:1084F80009062143596100780F2101400A439A6116
:10850800054A5A60054B1B6FDA02FBD4012010BDE7
:10851800FC000E408080000081DF000000000E405B
:108528002B4980230A6F5B0030B51A4201D1002025
:108538004DE0CB66274B02229C6C14420CD19C6CFC
:108548000422144207D19C6C250705D49A6CD406E2
:10855800EDD5052200E003229B24240214435C622B
:108568000C6FA502FCD4DC6A1A49240EC473DC6AB9
:10857800240C8473DC6A240A4473DC6A04739C6ADE
:10858800240EC4729C6A240C84729C6A240A447265
:108598009C6A04725D6B8024E4052C4005D001249C
:1085A8004470496B8903890B03E04470496BC90027
:1085B800490D41609C6B0F212140017000218170A1
:1085C800842149019963044901200A435A6230BD54
:1085D80000000E40FC000E408090000008B501200D
:1085E80004F0CCF8054804F0DBF803200021012250
:1085F80004F0DCF804F0FEF808BDC046409C00001A
:10860800364BF0B51A6801321A60354B1A680132D8
:108618001A60344B1A68002A02D01A68013A1A60A4
:10862800314B1A68002A08D01A68013A1A601B6888
:10863800002B02D12D4B01221A702D4B2D4C9B6A19
:108648009BB223602C4B21681A68914218DD206880
:108658002A491A682A4D801A2A4A884206DC28685C
:10866800696827681E681368BE1B2CE0286869685B
:108678001F68266813688022BE1B5202B61811E0D4
:1086880021681A68914225DA18681C4922681C4D2D
:10869800801A1C4A88420DDC286869681F682668A9
:1086A8001368BE1B5E43321CF317801A9941286079
:1086B80069600FE02868696827681E681368802267
:1086C800BE1B5202B6185E43321CF31712184B41F8
:1086D8002A606B602268084B1A60F0BD1C020020FB
:1086E800F4030020B0090020B4090020B8090020D4
:1086F80000000C403408002028090020FF7F0000FB
:10870800700800206C080020014B18687047C046AC
:108718001C020020704710B5FFF7F6FF074C2368CE
:10872800C01AFA235B00984207D9054B80215A6B7F
:108738004A409A62FFF7E8FF206010BDBC0900209C
:108748000010054010B5124CA378022B1CD86821E4
:10875800002001F07DFEA3784022FF329B010240F9
:108768001A430020682101F0F7FB2279E37812020E
:108778001A43637900201B041A43A3796A211B0654
:108788001A4301F0E9FB02E0024B04221A7010BD03
:10879800DC020020F803002008B50F4B58780028A9
:1087A80010D0012814D11A79D97812020A435979BC
:1087B8009B7909040A431B061A4300206C2101F027
:1087C800CBFB08E06C2101F043FE044B586002E04B
:1087D800024B03221A7008BDDC020020F8030020B7
:1087E800704770477047704770477047010C70B505
:1087F800C9B2051C00220120FBF75CFE0A4C290ABD
:108808000602C9B2002201202660FBF753FE064388
:108818000120E9B23602021C2660FBF74BFE064334
:108828003609266070BDC0462002002010B52A4CCB
:10883800C00023181A79032A01D903221A712318B0
:108848009A790433032A01D903229A7023181A7AD1
:1088580004330F2A01D90F221A7123185A7A0433C4
:10886800072A01D907225A7123189A7A04330F2A42
:1088780001D90F229A71221813798021DB03090389
:108888001943E1605279002A03D08422120313436A
:10889800E3602318DB79002B04D0E26880239B0176
:1088A8001343E36020188279037AD202DB01134371
:1088B800E26804301343427912011343E360C2793A
:1088C800002A02D182791343E360E068FFF78EFF44
:1088D800E368236110BDC0462002002010B5124C89
:1088E8000023C000E36023185B7E002B02D08023A6
:1088F8009B00E36023189B7E002B04D0E268802352
:108908005B001343E3602318DA7E14330F2A01D97E
:108918000F22DA712018E368C07E1843E060FFF781
:1089280065FFE268E26110BD200200200721414393
:1089380038B51E4C631C59180A1C1F325578CB7F5A
:108948002D039B03E0212B4309031943E16092782F
:10895800012A02D1164A1343E36007224243A218B0
:108968002032D378E1681B020B43E3601279012AB5
:1089780002D180221343E36007234343E3182033E3
:108988005B79012B03D1E26840231343E36007239B
:108998005843201820308079E36800011843E060CC
:1089A800FFF724FFE168A16238BDC046200200201D
:1089B80000040E00032310B543431F4C221C2C3225
:1089C800D31801229A563F2A01DD3F225A70032309
:1089D8004343221C2C32D31801229A563F3201DA23
:1089E800C1225A7003234343221C2C32D3189A788D
:1089F8001F2A01D91F229A700322C02342431B0356
:108A0800E360231C2C33D35C012B02D1D0231B033E
:108A1800E36003225043231C2C331B18E268987828
:108A280010435A787F2313401B021843E060FFF776
:108A3800DDFEE368236310BD2002002038B505225F
:108A4800264C4243231C3433D15C012901D901212E
:108A5800D15405234343221C3432D3185A78032AAD
:108A680001D903225A7005234343221C3432D318F8
:108A78009A780F2A01D90F229A7005234343221CA2
:108A88003432D318DA78032A01D90322DA7005239D
:108A98004343221C3432D3181A790F2A01D90F22E2
:108AA8001A7105235843221C343213181D79A0214A
:108AB800825C09032943081CD20310435A785203E5
:108AC80010439A78DB78120210435B011843E06088
:108AD800FFF78CFEE368E36338BDC0462002002040
:108AE80038B51F4B05211A1C01252C325170917085
:108AF800157003205A19D07752190024D0771A1804
:108B0800D4771A1DD4775A18D4779A1DD5770225A9
:108B1800DA1DD5771A1C3432997214705470947017
:108B2800D47014711D711D725C769C76DC765C7154
:108B3800DC719C715872DC7280220A4BD2031A6372
:108B4800201CFFF77BFF201CFFF734FF201CFFF7DA
:108B5800EDFE201CFFF7C2FE201CFFF767FE38BDA4
:108B68002002002000100540064A08B5C300D318AB
:108B7800D9761433042901D000225A71FFF7AEFECA
:108B880008BDC04620020020064A08B5C300D31815
:108B980059761433002901D00422DA71FFF79EFEBA
:108BA80008BDC0462002002008B5034AC300D318F8
:108BB8009976FFF793FE08BD20020020024BC00003
:108BC8001818C07E7047C04620020020024BC00023
:108BD8001818407E7047C04620020020024BC00093
:108BE8001818807E7047C0462002002008B5034A46
:108BF800C300D3181971FFF719FE08BD2002002021
:108C080008B5034AC300D3185971FFF70FFE08BD12
:108C18002002002008B5034AC300D318D971FFF712
:108C280005FE08BD2002002008B5034AC300D3187A
:108C38009971FFF7FBFD08BD2002002008B5034A23
:108C4800C300D3181972FFF7F1FD08BD20020020F8
:108C580008B5034AC300D3185972FFF7E7FD08BDEA
:108C68002002002008B5034AC300D3189972FFF701
:108C7800DDFD08BD20020020024BC0001818007955
:108C88007047C04620020020024BC00018184079E7
:108C98007047C04620020020024BC0001818C07957
:108CA8007047C04620020020024BC0001818807987
:108CB8007047C04620020020024BC0001818007AF6
:108CC8007047C04620020020024BC0001818407AA6
:108CD8007047C04620020020024BC0001818807A56
:108CE8007047C04620020020052208B54243034BC6
:108CF8003433D154FFF7A2FE08BDC046200200203D
:108D08000522424308B5034B34339B185970FFF7CB
:108D180095FE08BD200200200522424308B5034BFA
:108D280034339B189970FFF789FE08BD2002002094
:108D38000522424308B5034B34339B18D970FFF71B
:108D48007DFE08BD200200200522424308B5034BE2
:108D580034339B181971FFF771FE08BD20020020FB
:108D680005235843014B3433185C70472002002018
:108D780005235843024B3433181840787047C046CF
:108D88002002002005235843024B343318188078FA
:108D98007047C0462002002005235843024B343355
:108DA8001818C0787047C046200200200523584391
:108DB800024B3433181800797047C046200200204F
:108DC800032208B54243034B2C33D154FFF7F2FD7D
:108DD80008BDC046200200200322424308B5034BC9
:108DE8002C339B185970FFF7E5FD08BD20020020C1
:108DF8000322424308B5034B2C339B189970FFF7A5
:108E0800D9FD08BD2002002003235843014B2C3311
:108E1800185C70472002002003235843024B2C3370
:108E28001818407840B270472002002003235843A6
:108E3800024B2C33181880787047C0462002002057
:108E48000722424308B5034B01339B18D977FFF734
:108E58006DFD08BD2002002008B507234343034ADF
:108E6800D31820335970FFF761FD08BD2002002098
:108E780008B507234343034AD31820339970FFF7F3
:108E880055FD08BD2002002008B507234343034AC7
:108E9800D3182033D970FFF749FD08BD2002002000
:108EA80008B507234343034AD31820331971FFF742
:108EB8003DFD08BD2002002008B507234343034AAF
:108EC800D31820335971FFF731FD08BD2002002067
:108ED80008B507234343034AD31820339971FFF792
:108EE80025FD08BD2002002007235843024B01330B
:108EF8001818C07F7047C046200200200723584337
:108F0800024B1818203040787047C04620020020D5
:108F180007235843024B1818203080787047C04602
:108F28002002002007235843024B18182030C0782D
:108F38007047C0462002002007235843024B1818E8
:108F4800203000797047C04620020020072358438C
:108F5800024B1818203040797047C0462002002084
:108F680007235843024B1818203080797047C046B1
:108F780020020020F7B5334D1E1C2B1C4033041C67
:108F8800185C0191171C042825D803F09FFC030ADC
:108F980011181F00201CFFF749FC2B1C403301222D
:108FA8001AE0201CFFF7C2FC2B1C4033022213E0FE
:108FB800201CFFF743FD2B1C403303220CE0201C30
:108FC800FFF7F8FC2B1C4033042205E0201CFFF7B8
:108FD80085FC2B1C403300221A5507235C432C19AF
:108FE8002034A379012B11D0002B02D0022B13D0EF
:108FF80020E0019A002A03D02A68930C019A137082
:10900800002F17D02A68930A3B7013E0002E11D066
:109018002A68930A33600DE0002E03D02A68D30B28
:109028005B013360089B002B04D02A685304089A1C
:10903800DB0E1370099B002B02D02B68099A137062
:10904800F7BDC0462002002008B5002807D1044B10
:10905800D87A002803D10122DA72FFF7E7FB08BDAE
:109068002002002008B5002806D1044BDA7A002A2D
:1090780002D0D872FFF7DAFB08BDC04620020020F4
:10908800F8B5072343430F4F041CFB1820339E7980
:10909800032E03D003229A71FFF748FC201CFFF728
:1090A80045FC3D682B0301D5074B1D43032E07D014
:1090B80007236343FF182037BE71201CFFF736FCD7
:1090C800281CF8BD200200200000F0FFF8B506AC0F
:1090D8002778064D07AC2678C4002D19EF752E7633
:1090E80029756A75AB75FFF7F9FBF8BD20020020FA
:1090F80000B5062814D80B4B03F0E8FB0406080A51
:109108000C0E10001B680AE0DB6908E01B6906E02A
:10911800DB6B04E01B6B02E09B6A00E0DB7A0B6010
:1091280000BDC04620020020F0B5B84B89B01A78BF
:109138001F1C002A05D1B64B7B60BB60FB60012376
:109148003B703C7C002C0AD1E0B2FBF779F83B1C61
:109158001133E0540134082CF6D101233B74272441
:10916800201C2738C0B2FBF76BF83B19163B1A785E
:1091780082421CD0221C1870213AA64B9200D35868
:10918800022B06D0032B0CD0012B10D100280ED0B7
:1091980007E000280BD1A04A115D012907D113551A
:1091A80005E09D4B1A5D012A01D102221A550134AE
:1091B8002F2CD5D1994CE369002B19D0984D2E78D6
:1091C800002E15D1FFF7A0FA964BE2691B68C01A6A
:1091D800C1174018484090420AD9301C01F090F855
:1091E800012001F08DF8022001F08AF801232B708C
:1091F800236A002B19D08C4D2E78002E15D1FFF73D
:1092080083FA8A4B1B68C01AC117236A4018484062
:1092180098420AD9301C01F073F8012001F070F867
:10922800022001F06DF801232B70814C237B002B69
:1092380000D081E2FFF768FAFA69801AC317C018EC
:1092480058400A2804DC7B4B5B6B5E0300D5F3E2D5
:109258007E1CF07F002800D08EE10A2100F01EFF5E
:10926800051CF07F01F07CF9E91768184840049064
:10927800002D23D1F17F082349011943C9B2281CC5
:1092880000F00CFF002819D1FFF73EFAF37F9A008F
:10929800BA185268801AC11742184A4005925A01F2
:1092A800A218908B0A2141430598884223DD917AC0
:1092B800181CFBF788F8F37F01211AE07B1CD87F84
:1092C8005D4AC300049E99588E4202D2D318197978
:1092D80002E04301E318597A7E1CFBF774F8F27F29
:1092E8000592FFF711FA05998B00FB185860F37F78
:1092F8000021524AD154524E0499F07F4E4EC30079
:109308009B5999420BD2FFF751FD4D4AD37FDA00A2
:10931800B618727982420ED1181C002109E0FFF7B5
:1093280045FD4749CB7FDA00B6187179884202D0EB
:10933800181CFFF709FD7E1CF07F424B8200D318F2
:10934800414A002182180092404A821801920A1C60
:10935800FFF710FEF07F4301E3189B69002B17D03D
:10936800FBF738F8002813D0F07F049A4301E3187C
:109378009B699A420CD900F0C3FFF37F344A01215C
:10938800D154254A0F33D15C012901D10221D1548E
:10939800002D06D07B1CDE7F2E4B9B5D002B0BD156
:1093A8005CE07B1CD97F082349011943C9B2281CFA
:1093B80000F074FE0028EDD17B1CDB7F5A01A21857
:1093C800D289002A03D1234AD35C002B4BD0FFF764
:1093D8009BF91B4EF37F9A00BA18526A801A5A01F9
:1093E800C117A2184018D28948400A214A4390421E
:1093F80039DD194EF25C002A35D1181CFFF724FE1E
:109408000F4AD37F0122F2542DE0C04664020020A7
:10941800FFFFFF7F2C0900207E09002008000020A4
:10942800730900206C09002020080020640900202E
:10943800C8080020001005403C08002075090020DD
:10944800650200205C08002038080020C3080020BE
:10945800C0080020780900207B090020FFF754F994
:10946800B600BE197062CD4EF27F510163185B6978
:10947800002B00D180E0CA4B9E5C002E7CD1002DD1
:109488007AD002200143C9B2301C00F0E1FFC34981
:10949800051CC87F01F072F9C04A2D1AD17FE81760
:1094A8004B01E3185B692D184540D8171A1842403C
:1094B800954261DD002B27DD081C00F021FFB7492C
:1094C800CB7F5B01E3189B7F002B0CD17B1CDB7FE0
:1094D800B44A1533D15C012947D10221D15444E063
:1094E8000136032EF2D07B1CDA7F73015201A218D9
:1094F800E318927F9B7F9A42F2D1301C00F000FF64
:10950800F0B200F063FCEBE7301C022200F0DAFD59
:10951800A24A0823D17F301C49011943C9B200F07F
:1095280093FD9E48C37F5B01E3189B7F002B1CD0F3
:109538007B1CDA7F73015201A218E318927F9B7F8C
:109548009A420FD1F5B20020291C022200F0BAFD80
:109558006B01082119430020C9B200F075FD281CD1
:1095680000F034FC0136032EE2D17B1CD87F8C4CF2
:109578000123235400F02AFC002000F076FD3B1C58
:1095880030331A7807216E468A4301213076084223
:1095980000D00A431A70410705D53B1C30331A78AE
:1095A80002210A431A70C20605D53B1C30331A78CB
:1095B80004210A431A703B1C30331B787A4A0593FE
:1095C8007A4B11781B789C46794B1E78794B187822
:1095D800794B1D780023341C01221C41144213D0FE
:1095E800059C1C4114420FD00C1C1C4114420BD189
:1095F800151C9D40EDB2294328436446C9B2C0B248
:10960800151C002C00D166460133032BE3D1664BB1
:10961800674A1970674B16701870674B01221D70E6
:109628003B1C30331B7813420AD0391C313109787E
:10963800114205D15B4AD178012901D10221D170AB
:109648000222134209D0391C31310978114204D160
:1096580054490879012800D10A71042213420AD01A
:10966800391C31310978114205D14E4A5179012905
:1096780001D1022151717D1C3A1CEE7F31321370E9
:10968800301C032103F036F906ACC0B2235C7F2BF3
:1096980043D97601162107AC3143C9B20020221CF8
:1096A80000F0EAFCA3785E0608D5EA7F3D4952003F
:1096B8001B32885C012801D1022088545AB2002A42
:1096C80009DA7A1CD27F37490E325200885C0128A9
:1096D80001D102208854D80609D57A1CD27F314995
:1096E80052001B32885C012801D102208854990657
:1096F80009D57B1CDB7F2B4A0E335B00D15C01292B
:1097080001D10221D1547B1CD97F16234901194369
:10971800C9B20020221C00F0F5FB7C1CE07F00F0A1
:109728008DF8E37F0133DBB2032B00D90023E37705
:10973800FEF7EAFFF8617FE0204D214B00227E1CF6
:10974800F277101C00930195111C1E4BFFF712FCB9
:10975800F07F3B1C2A5C32331B4D1B5C7F2A35D8BB
:10976800022B02D12B5C002B0FD04301E418617A45
:109778007C1CFAF728FEE07FFFF774FCE37F3A1CB5
:1097880032320221D1540022EA547B1CDC7FFEF7DE
:10979800BBFFA4003C1960604EE0C0466502002093
:1097A800570800207E0900203108002030080020DA
:1097B8005B0800205A080020AD090020C3080020DB
:1097C800380800205C08002070090020012B05D112
:1097D8007B1CDB7FEB5C002B11D12DE0FEF794FFA7
:1097E800F37F9A00BA1852685B01801AC217E3180F
:1097F80080189B8B50400A2253439842E8DD7E1C18
:10980800F07F4301E318997AFAF7DDFDF07F430111
:10981800E418A37A002B02D1FFF716FC04E02B5CB6
:10982800002B01D0FFF71EFC7B1CDB7F3A1C323279
:109838000121D1540022EA5409B0F0BDF0B5041C4E
:10984800400189B0C7B27C210190394307AA0020A2
:1098580000F012FC610004916A46937F02228A405C
:109868001A40029201228A40134001980593D04B76
:109878007F211A18127A0020114052B20391002A4F
:1098880004DAFAF7DDFC4642464104E0FAF7D8FC70
:10989800061C701E86410398F6B20138072800D9C5
:1098A80084E2C44D03F01CF8080008000800080012
:1098B8003F013F013F013F01285D0F2800D975E2B4
:1098C80003F00EF8740210003600460054006400DD
:1098D8006D007C009200C200FA00FF0074021E01B5
:1098E80027015E021421394307AA002000F0C4FBB7
:1098F80069464B7FA600AE19736006231F43391CC7
:10990800002000F0CBFB211C30610222002000F077
:10991800D9FB0020391CA84A00F010FB0020211CAC
:10992800032200F0EBFB039B023B012B1CD893E1C5
:10993800A300EB185A6804231A4001231A43002095
:10994800211C00F0DBFB08213943994B019843E1C6
:109958000599002900D129E202213943002000F0AD
:1099680077FD964BA200D05004231EE2A300EB180B
:109978005A6804231A4002231A430020211C00F0CD
:10998800BDFB082139438A4B019854E1029900290B
:1099980000D10BE2201C00F0B3FC062305E2211CD9
:1099A8000020032200F0AAFB0198814A082113181D
:1099B80039435A68002000F0C1FA54E1029900299D
:1099C80000D0F3E10826081C3743021C391C00F0BC
:1099D800B5FA774A0198391C13185A680298524206
:1099E80000F0ACFA2E55E1E10299002900D1DDE141
:1099F80002213943002000F02BFD0821061C00201D
:109A0800021C394300F09AFA6C4BA200D058811B13
:109A1800D1500020211C032200F070FB644A0198F9
:109A2800062113185A683943002000F087FA019A72
:109A38000020D1B2321C00F08FFA0020211C021C39
:109A480000F040FB0923B0E1002000F00EFB049B6E
:109A58001841C10700D4A9E1082500203D43021C94
:109A6800291C00F06BFA02260020211C022200F0BB
:109A780029FB0020311C3943021C00F06DFA019AC1
:109A88000020D1B2021C00F067FA039B494F033B48
:109A9800012B0FD80020211C321C00F013FB444876
:109AA800019943185A6800205242291C00F046FACE
:109AB8000A2342E10E2340E1029A002A00D015E170
:109AC80074E1029B002B00D070E10221181C39437D
:109AD80000F0BEFC061C02980821021C394300F065
:109AE8002DFA0198F20F9619C1B27210029800F07F
:109AF80033FA0298211C021C00F0E4FA0D2354E109
:109B0800002000F0B2FA04990841C20700D542E1EA
:109B18004CE1A600AE19062132693943002000F055
:109B28000DFA32793CE1285D0F2800D93EE102F0B8
:109B3800D7FE3D01100032005900690089003D013F
:109B48009C003D013D01D300DF00B5000601340152
:109B580027011421394307AA002000F08DFA68462E
:109B6800427FA300EB185A600020211C022200F05B
:109B7800A9FA0621394300200F4A00F0DFF9211C19
:109B88000020032200F0BAFA0399062964D00829B4
:109B980000D0E9E660E0039A062A11D1A300EB1889
:109BA8005A6804231A4001231A430020211C0DE09F
:109BB800C80800209C020020FF070000240800209D
:109BC800039B082B04D10020211C032200F096FAE5
:109BD80008217748019B3943C258002000F0AEF9AC
:109BE8000323E2E0039B053B012B06D805980028D8
:109BF80003D00399062931D1B6E60C23002E00D0F4
:109C0800D3E0D3E0039A052A09D1A300EB185A68D8
:109C180004231A4002231A430020211C05E0039B59
:109C2800072B04D10020211C032200F067FA082129
:109C38005F48019B3943C2580020524200F07EF928
:109C48000523B2E0039B053B012B09D802980028A5
:109C580006D00399052901D10223A6E00F23A4E029
:109C6800002E00D1A2E007239FE0002E00D09DE047
:109C7800039B073B012B0AD9A300EB185A6804235E
:109C88001A4001231A43301C211C00F037FA484AB5
:109C980001980821131839435A6818E0002E00D09B
:109CA80084E0039B073B012B0AD9A300EB185A68F1
:109CB80004231A4002231A43301C211C00F01EFA08
:109CC8003B4A0198082113185A6839435242002028
:109CD80000F034F90A2368E0002E67D002213943E6
:109CE800002000F0B5FBA300EB18D8610B235CE063
:109CF800002E5BD102213943301C00F0A9FB2C490E
:109D0800019A051C8B18062139435A685E73301C6A
:109D180000F022F9019B274FD9B2A300FB18DB6999
:109D2800301CED18EA0F55196A1000F015F9301CAF
:109D3800211C321C00F0C6F90D233B5536E00020EB
:109D480000F093F904990841C2072FD50020082193
:109D58000E233943021C2B5500F0F0F8211C00207B
:109D6800022200F0AFF9002002213943021C00F062
:109D7800F3F8019B0020D9B2021C00F0EDF815E0C1
:109D88000020211C022200F09DF9082100203943FF
:109D9800021C00F0D3F80E2307E0A300EB181A7991
:109DA8000020211C00F0AAF900232B5509B0F0BDB2
:109DB800C80800209C020020034B1A5C002A01D12D
:109DC80001221A547047C0469C020020034B1A5CBB
:109DD800002A01D00F221A547047C0469C02002066
:109DE800014B185C7047C0469C0200200000000030
:109DF800F7B51378071C5D060E1C141CAD0F27D190
:109E08003A496A018A18117B0832002920D1D907FA
:109E18001ED45F2B1CD83649495D002918D168210A
:109E28008B43019314D133494B5D002B06D05178F5
:109E38000198FAF7C8FA019B2E4A53552E494B5DF3
:109E4800002B05D00020FFF70DF92B4A00235355AE
:109E580000202178021CFAF72DFB30700020617871
:109E6800021CFAF727FB70700020A178021CFAF791
:109E780021FBB070E17800200122FAF71BFBF0709B
:109E88002378D90731D45F2B2FD81E221340082BF3
:109E980010D0142B20D0062B27D10C235D4324236C
:109EA8005F43A378ED19E278144F1B027D19134321
:109EB8006B601AE00C2045432420A1784743E278E0
:109EC800090211430D4AED19A950A07818420CD087
:109ED8000B4B1943A95008E00C2255432422574341
:109EE800ED19064FE3787D192B72F7BDC8080020DD
:109EF80078090020750900207B09002078080020D7
:109F080000F0FFFF07B56B461970137869464B7070
:109F180053788B7093786A46CB7001A9FFF768FF76
:109F280007BD37B506AC6D46247829706A7001A95B
:109F38006A46AB70EC70FFF75BFF37BD07B56B4641
:109F48001970694600234B701312CA708B706A46E9
:109F580001A9FFF74DFF07BDF0B5051C85B00E1C24
:109F6800141C5F295BD81E2248060A40800F019204
:109F7800002A02D0022A20D051E0032169432F4F42
:109F88000918090178184368CC510091E11ACA17D9
:109F9800891851408C46391C294FBC450ADD9C4222
:109FA80001DDDC1901E0274A9C18009BC918012330
:109FB8000B7334E00199017331E003276F431F4BA2
:109FC8003F183F01DA19111C083100912102090AD2
:109FD80091605460FA581A4B0192121BD11752180B
:109FE8004A409A4218DD174A0199A318A14201DD97
:109FF800134AA31869461A144A7240011A120872C1
:10A008008A72CB7202AA281C03A9FFF7F1FE0B4A39
:10A018000123D7193B7302E0009900230B716A46AC
:10A0280023145372231216729372D472281C03A934
:10A0380002AAFFF7DDFE05B0F0BDC046C00900204A
:10A04800FFFF7F00010080FF07B51C220A4002D1F4
:10A05800FFF782FF08E06A460023117001A95370D8
:10A068009370D370FFF7C4FE07BD08B50121002027
:10A078000A1CFAF71FFA08BD13B50123141C19436B
:10A0880001AA11706946FFF7B3FE6A465378107843
:10A09800237093786370D378A37016BD07B5012336
:10A0A800194301AA11706946FFF7A2FE6A46907823
:10A0B800D37800021843030501D5014B18430EBDA0
:10A0C80000F0FFFFF7B54E0101ACF6B21523171CDF
:10A0D80033436A46211C051C1370FFF789FE1423BD
:10A0E8001E436B461E7063786A465370A378281C1B
:10A0F800211CD7709370FFF77BFEF7BDF7B54E01B3
:10A1080001ACF6B21523171C33436A46211C051C03
:10A118001370FFF76DFE14231E436B461E706378A1
:10A128006A4697705370E378281C211CD370FFF798
:10A138005FFEF7BD73B501AC6A467F230E1C211C78
:10A14800051C1370FFF754FE6A467E23137063786C
:10A15800281C53700F231E409670E378211CD3707F
:10A16800FFF746FE73BDF0B5490587B0490D4001BC
:10A17800C0B2029105AE182103900143321C0020A1
:10A18800FFF77AFF73780F271A0900921F40029889
:10A1980097420EDB03F0A0FE009B041CFF1A01206F
:10A1A800B8400D1C03F05AFE304B2F4A03F092FBC7
:10A1B8000FE003F091FE009A041CD71B0120B84061
:10A1C8000D1C03F04BFE021C0B1C2849264803F00B
:10A1D8005DF8021C0B1C201C291C03F057F803F027
:10A1E80001FF03F0ADFE224A224B03F073FB03F09C
:10A1F800F9FE03F0A5FE204A204B03F06BFB012576
:10A20800009001916D422F1C00240120A04003F012
:10A2180025FE0B1C021C0098019903F05BFB03F060
:10A22800E9FD031C803B7F2B01D9381C00E0251C6D
:10A2380001340E2C01D0071CE7E7039B00241221F0
:10A2480019437070321C201C3470B570FFF75AFE29
:10A25800039A0C211143201C029AFFF76FFE201C61
:10A2680007B0F0BDC046C0460000000000006040D6
:10A2780004560E2DB29DEF3F000000000000204064
:10A28800F7B54B0803255D43B42343430135FF3538
:10A29800ED18071C281C0E1CFDF7D7FE01AC20701A
:10A2A800681CFDF7D2FE6070A81CFDF7CEFE790190
:10A2B8000E43A070F1B20020221CFFF723FEF7BD69
:10A2C80073B50D1C410101AC2943221C061CC9B2FF
:10A2D8000020FFF7D1FE6D0803235D43B4235E43DE
:10A2E8000135FF35AD19281C2178FDF7C7FD681C1D
:10A2F8006178FDF7C3FDA81CA178FDF7BFFD73BD0C
:10A3080010B5C4B20222211C00206401FFF7DAFE56
:10A31800E4B2082121430020FFF796FE0A212143D9
:10A328000020FFF791FE10BD73B5400116250543C7
:10A3380001ACEDB2221C0E1C0020291CFFF79CFE6C
:10A3480063784022F10701D5134300E0934363701B
:10A358001023B20702D56278134302E062789A4369
:10A36800131C0020291C221C6370A070FFF7CAFD73
:10A3780073BD73B540011625054301ACEDB20E1C43
:10A388000020291C221CFFF777FE6378F20703D50B
:10A3980080225242134301E07F221340637020233E
:10A3A800B20702D56278134302E062789A43131C1D
:10A3B8000020291C221C6370A070FFF7A3FD73BD49
:10A3C80013B540011621014301ACC9B20020221C7B
:10A3D800FFF752FE63785806C00FDA0601D502234C
:10A3E800184316BD13B540011621014301ACC9B28B
:10A3F8000020221CFFF740FE6378D8099A0601D591
:10A408000223184316BD70B5104E000133189A6820
:10A4180091420ADD80248A1A6404A41A5D68A24263
:10A4280001DCAA180BE02C1B0CE091420BDA80240B
:10A43800521A6404A41A5D68A24202DCAA1A5A607D
:10A4480001E02C195C603018816070BDC0090020E3
:10A4580037B501230B4301AA0C1C69461370051C70
:10A46800FFF7C6FC69464A788B7812041B0213432F
:10A47800CA78134380221204134202D0FF22120624
:10A4880013435F2C19D862061E21920F0C400ED080
:10A49800022C12D103214D431B025519E8B2190AA7
:10A4A800FFF7B1FF064B2D015D196B6805E003232B
:10A4B8005D43034BAA181201D358181C3EBDC04671
:10A4C800C009002038B50D1C6821041CFFF7C0FF27
:10A4D8000122002D01D0024301E09043021C201C00
:10A4E8006821FFF739FD38BD73B51B4B587E012332
:10A4F800184004D0242200206821FF3202E0912273
:10A5080068215200FFF728FD0020022300937E21D6
:10A51800021C031CFFF705FD00250024EEB2E1B282
:10A52800301C0134FFF7ACFE1D2CF7D17401E4B2E6
:10A538000C2121430020FFF78BFF011C301CFFF783
:10A5480012FE162121430020044A0135FFF7F6FCCC
:10A55800032DE2D173BDC04608000020FF31000082
:10A56800F0B587B004AD4601032305AA041C3343A4
:10A57800291C00201370FFF73BFC6978AB780904AD
:10A588001B021943EB78201C1943FFF73CFF174ABD
:10A5980021015318181C083003900579002D23D089
:10A5A8000C256C43124D2C19247A002C1CD18D5883
:10A5B8005B68EF1AF8173F184740BC460D4FBC457B
:10A5C80005DD0D4A98189D4204DDD81902E0039B69
:10A5D80088581C7102140312C0B20090F1B2D2B2B2
:10A5E800DBB20020FFF79DFC07B0F0BDC0090020DA
:10A5F80078080020FFFF7F00010080FFC046C046AA
:10A6080008B5164B0120D86299690F221140144AE7
:10A6180007290AD0082910D0062915D1186B114925
:10A628008860D9691160072205E0186B0D494860F8
:10A63800D969116008229A610BE0186B0949086012
:10A64800D96911600622F6E7D969116006229A6174
:10A65800D862024801F09AFA08BDC04600000440DA
:10A66800F0090020C402002013B5134C0621201C59
:10A6780001F05AFA201C072101F056FA201C082183
:10A6880001F052FA201C00231D21062201F066FA6F
:10A6980001210A1C201C01F07FFA01A80523037080
:10A6A80007234370002383700123C37001F008FF60
:10A6B800201C01F06BFA13BD00000440002302289F
:10A6C80002D8024B8000C358181C7047C4020020EF
:10A6D80010B50C490C4C00220023802048622260EF
:10A6E80063600A4A00231360094A1360094B1B7808
:10A6F800002B05D18B6983438B61CB681843C860F5
:10A7080010BDC04600000C40700800202809002039
:10A7180034080020F4090020002802D1014B090167
:10A72800196070476C080020002821D1114B802245
:10A73800480705D55A629A61D8689043021C04E01C
:10A74800986990439861D8680243DA600822C8067D
:10A7580002D5D868024302E0D8689043021CDA6048
:10A7680008231940044B02D001221A7000E0197026
:10A778007047C04600000C40F409002000229042B7
:10A7880005D1044B1A685B681B06120A1A43101C91
:10A798007047C0467008002070B5041C0D1C0028C6
:10A7A8001AD1F9F705FE2A1CEB170C4D2A606B60CD
:10A7B800286869680B02060E020233432A606B6040
:10A7C800074B08481C60084B1C6001F013FC054847
:10A7D80001F015FCF9F7EAFD70BDC04670080020CD
:10A7E8003408002000000C402809002037B500205C
:10A7F8001E21032201F096FD00201F21032201F0F3
:10A8080091FD164C01200021032201F08BFD01254A
:10A8180000216560201CA5600A1C01F0C3FBE368E9
:10A8280080221343E3600E4B0E4A1B69002059092E
:10A83800090111601F211940FFF776FF0020011C54
:10A84800FFF7AAFF01A80923037007234370002319
:10A85800C570837001F034FE37BDC04600000C405F
:10A86800C80800206C08002070B51E4E3368DA0155
:10A8780037D433689A0134D41B4C6368A2689D1A94
:10A88800102D00D9102500202A1C031CE16800F0B7
:10A89800D3FCE2685319A268E360AB186268A3604E
:10A8A800934219D13268802040040E4B10400DD1DC
:10A8B8001968102D06D1802292040A431A6000F00C
:10A8C80089FC03E0A02212050A431A600023E36012
:10A8D800A3606360236004E0326880239B04134311
:10A8E800336070BD20001040000A00200E4B1A1C77
:10A8F80062321278002A06D0012A0DD1996E0222FE
:10A908000A439A6608E01A1C643211787F220A40CA
:10A91800013212010121D150044B90221968D2054D
:10A928000A431A607047C046000A00202000104001
:10A9380010B5224A131C62331878214B002806D020
:10A94800012834D1906E0221884390662FE0111CB3
:10A9580064310C787F2121404C1C2401A05012192D
:10A968005268002A0ED1002902D11968154A0DE053
:10A978001548164A09188900086802400A600868DC
:10A98800134A12E00F4A002907D119680A401A60D1
:10A998001968104A0A401A6009E00B48091889002A
:10A9A8000C680D4820400860086802400A60196871
:10A9B8009022D2050A431A6010BDC046000A002042
:10A9C80020001040FFFFFFDF08000410FFFFDFFF3B
:10A9D800FFFFBFFFFFFFFFFBFFFFFFEF08B5304B97
:10A9E80080211A1C63321078C9052E4A022816D015
:10A9F800032828D0012845D11068014311601A1C8A
:10AA08006732191C12786631097812020A43122A31
:10AA180000D912225A6000229A60234A2CE010685A
:10AA2800014311601A1C6732191C127866310978C3
:10AA380012020A43092A00D943225A6000229A6066
:10AA4800194A123218E0106801431160191C673165
:10AA58000878191C1A1C66310978623212780002CB
:10AA68000843114992008A18926D586011788842FB
:10AA780000D9596000219960DA6001221A60FFF755
:10AA8800F3FE0CE0106880239B05034313601368F2
:10AA9800194311601168A0231B050B43136008BDFF
:10AAA800000A00202000104074E3000008B5534A53
:10AAB800131C6033197807231940131C01291ED071
:10AAC800002902D002296ED097E061321078092857
:10AAD80020D801F0FBFE45751F721F05901F4D26FB
:10AAE8001A1C6232117880221143454A1160454A86
:10AAF80090211068C9050143116000220FE0131C62
:10AB080061331B780A2B40D00B2B3BD1131C6233CB
:10AB18001B7813673B4B90221968D2050A431A60C9
:10AB28006BE01A1C623212789021DA66354AC90540
:10AB3800106801431160344A3448910059180918C3
:10AB480009681068002902D18021090401E08021E8
:10AB5800C905014311602E4904328A42ECD14CE008
:10AB6800284A80211068C90501431160996E06E0E2
:10AB7800244A80211068C90501431160D96EC9B201
:10AB8800244B31E0062B38D135E01E4B8021186864
:10AB9800C90501431960116F1E4AC9B21160A0228C
:10ABA80019681205BAE761321078062825D801F02D
:10ABB8008DFE0A07240424242200FFF797FE1CE0D8
:10ABC800FFF7B6FE19E00F4A80211068C905014356
:10ABD8001160191C643108787F2101400131090195
:10ABE800595C0C4B1960002119601168A0231B05E2
:10ABF8000B43136001E0FFF7F1FE08BD000A0020D7
:10AC080000001040200010402400104094FFBFFFB7
:10AC1800340010408000104008B500F02FFC0028D8
:10AC28000CD1074B60331A7807231340012B05D149
:10AC3800044B90221968D2050A431A6008BDC04621
:10AC4800000A00202000104010B5274A00280AD129
:10AC5800264B19684C0117D5186825490140196019
:10AC6800186824490BE0244943189B0019684C02D2
:10AC78000AD518682149014019601868204901401F
:10AC88001960002313602EE01B4943189B001968C4
:10AC9800CC0006D51C6880210906214319600021D3
:10ACA80011601268002A04D0012A1CD1FFF7DCFDCC
:10ACB80019E001221B68002801D11B0E00E01B0CC3
:10ACC800134010D00F4C08220023211C00F0A4FAD6
:10ACD80022786023134004D0202B04D1FFF79CFF77
:10ACE80001E0FFF7E3FE10BD000A0020200010403D
:10ACF800FFFFFFDFFFFFFFFB08000410FFFFDFFF80
:10AD0800FFFFBFFF600A0020704708B500F010FE83
:10AD180008BD08B500F0E6FD08BDC04608B5011C31
:10AD28000822024803F0A6FA002008BDD00200203D
:10AD380008B50249082203F09DFA08BDD002002098
:10AD480070477047704710B5094B962292011A60F8
:10AD5800002408221C715C719A71064B0122524230
:10AD68001A60FFF7D2FF00F0A5F9201C10BDC046FD
:10AD7800D0020020480000200020704710B5054C84
:10AD88002368002B04D0022000F0D6FD00232360A6
:10AD980010BDC0464800002073B56E460736051C36
:10ADA800301C00F051FE002801D100201AE00E4BA3
:10ADB800307819780D4C4A1CD2B21A7060541E1C97
:10ADC800092AF2D10023E25CEA540133092BFAD1B3
:10ADD80000F032FE002803D0201C00F035FEF7E713
:10ADE8003070012076BDC046FE090020F50900201C
:10ADF800024B01211A688A431A607047B400104058
:10AE080008B501F0B8FC01F0B6FC01F0B4FC01F0A3
:10AE1800B2FC08BD08B501F0AEFC01F0ACFC01F0D5
:10AE2800AAFC01F0A8FC08BD0023834201D201233B
:10AE3800FBE7704738B50D1C111C141C01F09EFD72
:10AE48000120002907D1281C211C01F097FD081CAE
:10AE5800411E8841400038BD031C411800208B4228
:10AE680003D01A7801338018F9E770478900031C6A
:10AE7800411800208B4202D004CB8018FAE77047B3
:10AE88008218904202D001700130FAE77047000042
:10AE9800024B034A1360034A13607047FFFFFF0029
:10AEA800600010406400104038B50D1C0721041CD8
:10AEB80001F064FD8B005B421833062C01D90A4A65
:10AEC80000E00A4A12680F2199408A439D40111CEC
:10AED800802329431B061943062C01D8034A00E0A6
:10AEE800014A116038BDC04664001040600010403F
:10AEF80030B50F49441C25014D196A60002B02D05A
:10AF080005014D192B772401002A01D10A5103E0CC
:10AF1800012380220B5192010649431806498000FB
:10AF280041588020C90801439B000A431A6030BD7C
:10AF3800000A00200800041064E4000038B51E4D23
:10AF480000217822281CFFF79BFF281C00210822DB
:10AF58006030FFF795FF194A194B0024AC661A6058
:10AF6800FFF796FF0120211C80220323FFF7C0FF73
:10AF78000220211C221C0323FFF7BAFF114BA20059
:10AF8800E358AA18402B00D9402304349361142CA9
:10AF9800F4D10D4B88211A680A431A600B4B012122
:10AFA8001A680A431A600A4A0A4B1A600A4B0022B6
:10AFB8001A60FFF7AEFE38BD000A0020820000C00C
:10AFC8002000104064E40000A0001040B4001040CD
:10AFD8007F0400000C0010400400104070477047C8
:10AFE80038B51C4B02019A18117F421C12019B189C
:10AFF8005A68002A0CD100280CD0174C03199B0062
:10B008001C68650216D51968144A0A401A601FE0C0
:10B01800002806D1124B1C6865010BD51968114A26
:10B02800F3E70D4C03199B001C68A50002D51968AD
:10B038000D4AEAE703290BD1032802D100F016FCD8
:10B0480006E0802A02D100F095FB01E000F020FB29
:10B0580038BDC046000A002008000410FFFFBFFFEB
:10B0680020001040FFFFFFFBFFFFFFDF104B10B574
:10B078001C681C60630501D5FFF760FFE30702D574
:10B088000020FFF7E1FDA30702D50120FFF7A8FF85
:10B09800630702D50220FFF7A3FF230702D5032089
:10B0A800FFF79EFFE30602D50420FFF799FF10BDC6
:10B0B800080010400B4A002353670B4A8820116888
:10B0C80001431160094A01201168014311600849D0
:10B0D800084A1160084A8021C9001160074A1360B4
:10B0E8007047C046000A0020A0001040B40010407D
:10B0F8007F070000080010400C00104004001040BA
:10B10800194A431C1B0101219950D3185B68002B75
:10B1180017D1002809D1154B8022196892050A43D6
:10B128001A6080221968D20511E0114BC0188000FE
:10B13800026880239B031343036002680D4B13408E
:10B148000FE0002806D1094B8022196892050A43AE
:10B158001A6007E0064BC0188000026880235B0570
:10B16800134303607047C046000A002020001040C7
:10B1780008000410FFFFFEFF094B04211A6882B083
:10B188000A431A60802252030192019A511E0191CA
:10B19800002AFAD11A6804218A431A6002B070475B
:10B1A80004001040002806D1074B80221968D205F8
:10B1B8000A431A6006E0054BC01880000268044B79
:10B1C800134003607047C046200010400800041078
:10B1D800FFFFFEFF10B50E4943189B00002808D159
:10B1E8000C4A11688C010DD50A4A1268D401F5D5AC
:10B1F8000DE08022196852041142F5D119680A43FA
:10B208001A6004E01168A0231B050B43136010BDEE
:10B218000800041020001040002A09D0054B8A18A5
:10B22800C0188000914203D003680B700131F9E720
:10B238007047C04620000410002A09D0054B8A1820
:10B24800C0188000914203D00B7801310360F9E700
:10B258007047C04620000410F0B585B00192204A1E
:10B2680000268718041C02910393BF00351C019A1D
:10B2780096422AD20123002C03D11A4A1268520E90
:10B2880001E03A68120E9343F4D0174A2301D31809
:10B298009B69019A951B9D4200D91D1C029B201C8D
:10B2A80099192A1C039BFFF7C7FF7619002C06D1B2
:10B2B8000C4B8022196892040A431A60D7E73A684F
:10B2C80080235B0413433B60D1E7074A2301D3186B
:10B2D8009B699D4202D1201CFFF77CFF05B0F0BDA1
:10B2E8000800041020001040000A0020F0B5384B78
:10B2F80095B01A680291411C8A4301911A60354A37
:10B30800041C8618B600311C2031039100250299CF
:10B318008D424FD2304B621C12019A185268191C88
:10B328000123802A24D1002C03D12C4A1268520E02
:10B3380001E03268120E9343E9D022018B189B6911
:10B34800029A571B9F4200D91F1C201C04A93A1CB3
:10B358000123FFF771FFED19002C04D11F4B802248
:10B36800196892041EE0326880235B0413431FE0CF
:10B37800002C03D1194A1268120E01E03268120C2F
:10B388001340C4D0039B201C1F6804A9FFB23A1CB9
:10B398000123FFF741FFED19002C06D10F4B802246
:10B3A8001968D2050A431A60B1E732680C4B13409A
:10B3B8003360ACE7019B01229A400A4B04491A60AA
:10B3C8000B68019A281C13430B6015B0F0BDC046EA
:10B3D8000C00104008000410000A00202000104053
:10B3E800FFFFFEFF0800104070B5204B451C2A01E6
:10B3F8009C1866681C1C802E04D1002920D00129C5
:10B408001ED032E001291BD0002902D0022919D010
:10B418002BE0D358012B0FD1002806D1144B8022E2
:10B428001968D2050A431A6006E0124BC01880005A
:10B438000268114B134003602D010023635114E08F
:10B44800D15012E0D358002B0FD1002806D1084B59
:10B4580080221968D2050A431A6006E0054BC01815
:10B4680080000268044B1340036070BD000A00208E
:10B478002000104008000410FFFFFEFF73B5804B4A
:10B4880000241A1C653211781A1C643212780902D9
:10B49800114309B2A14200D0F0E01A1C60321478BE
:10B4A80007221440012C00D0D5E01A1C6132127812
:10B4B800202A50D004D8002A0AD0012A35D0CCE05E
:10B4C800222A00D194E066D3232A00D1A5E0C4E063
:10B4D800191C6331181C097862300078090201438D
:10B4E80057D1191C6731097866331B7809020B4359
:10B4F800072B4ED8634A80211068C90501431160A3
:10B508001168C801FCD5013B5F499BB28B4205D04D
:10B518005E4968460968C9B20170F4E7116890236A
:10B52800DB050B431360012233E0181C63300078FD
:10B5380062331B78000203430BD1524B80211868F9
:10B54800C905014319601868A0210905014319605C
:10B558001FE00A1C1DE01A1C6332181C12786230A6
:10B5680000781202024312B2002A74D1191C673102
:10B57800097866331B7809020B43072B09D1414A26
:10B5880080231168DB050B4313601368D901FCD5D0
:10B5980065E0141C72E01A1C633215781A1C6232BA
:10B5A80012782D0215432DB2002D54D11A1C673282
:10B5B800127866331B7812021343072B16D1314ECB
:10B5C80080233268DB05134333606846FFF7B0FB1E
:10B5D8002B1C6A46D15C2D4A01331160072BF8D128
:10B5E8003268A0231B051343336047E02C1C45E059
:10B5F8001A1C6732181C127866300078120202434F
:10B6080029D11D1C6235287840082040FFF798FB97
:10B6180028782040FFF795FB16E01A1C6732181CA3
:10B628001278663000781202024314D11A1C633271
:10B63800107862331B7800021843134B984201D1EB
:10B6480001204042FFF77EFB0E4B90221968D2057D
:10B658000A431A6012E00C1C10E000240EE00023DC
:10B668000A496846096819540133072BF8D111684B
:10B678009023DB050B431360FFF750FB201C76BDBE
:10B68800000A002020001040FFFF0000800010404A
:10B69800F0B5051C85B0002803D1314B1A68120E8D
:10B6A80004E030482B189B001A68120C01239343BE
:10B6B80001930199002951D12B4AAB189B000393A0
:10B6C8001B68DFB2002F03D1281CFFF76BFD45E094
:10B6D800264C84239B00E35880204000C31A9F42D5
:10B6E8003CDC8526B600A159421A09180292611855
:10B6F800281CBA420EDB01233A1CFFF78DFDA05926
:10B7080080213B1849008B4201D0A35112E0019AD5
:10B71800A2510FE0029A0123FFF77EFD029B611CF4
:10B72800FB1A0193281C1A1CFF310123FFF774FD33
:10B738000198A051002D05D1094B80221968D20526
:10B748000A4304E0039B0A4A203B19680A401A602E
:10B75800064A84239B00D058C119D15005B0F0BDCA
:10B76800200010400800041010000410780A00207F
:10B77800FFFFFEFFF7B5051E03D1394B1B689B0180
:10B7880004E0384A83189B001B68DB01DB0F66D195
:10B79800354C80239B00E658002E19D183239B004B
:10B7A800E15C1A1C00295AD0002D06D12C4B8021AF
:10B7B800186889040143196007E02A4BED18AD00A9
:10B7C800296880235B040B432B600023A35446E0C5
:10B7D800402E00DD402682239F00E159802252003E
:10B7E800521A01926118281CB2420CDB321C012348
:10B7F800FFF722FDE259B31880225200934200D18C
:10B808000023E3510EE0019A0123FFF715FD019B88
:10B81800281CF31A1A1C0193211C0123FFF70CFDA5
:10B82800019AE251002D06D10D4B8022196892042D
:10B838000A431A6007E00B4BED18AD002A68802315
:10B848005B0413432B6083239B000122402E00D00E
:10B858000022E25480239B00E258961BE650F7BD75
:10B868002000104008000410780A002038B5041E93
:10B8780003D1184B1B689B0104E0174A83189B00EF
:10B888001B68DB01DB0F23D1144D88229200AA5CD0
:10B89800002A1DD087229200AA581149201C0A723A
:10B8A8000A22FFF7C9FC002C06D10A4B802219682E
:10B8B80092040A431A6007E0074BE418A4002268C0
:10B8C80080235B0413432360882300229B00EA54EF
:10B8D80038BDC0462000104008000410780A002037
:10B8E8004C00002008B58021104B002289005A50D6
:10B8F800812189005A50822189005A508321890068
:10B908005A54842189005A50852189005A50862129
:10B9180089005A50872189005A50882201219200B3
:10B9280003209954FFF7A2FF08BDC046780A0020FB
:10B9380008B5FFF7D7FF08BD08B58722074B920067
:10B9480098508822012192009954F8F7BBFB0320F4
:10B95800FFF78CFFF8F7B4FB08BDC046780A002053
:10B96800034A80239B00D35880204000C01A7047A8
:10B97800780A002010B580230F4C9B00E3588021E3
:10B9880049008B4216D081239B00E258A054013213
:10B998008A4200D10022E250F8F794FB80239B00F2
:10B9A800E25801200132E250FFF7E4FEF8F788FB85
:10B9B800012000E0002010BD780A0020F7B58023A0
:10B9C8001C4C9B00E358802701907F000020FB1A45
:10B9D80083422ED00D1E9D4200DD1D1C8126B6001F
:10B9E800A05901993F1A2018AF420BDB2A1C02F01C
:10B9F80041FCA15980226B185200934200D10023C8
:10BA0800A35109E03A1C02F035FC019BEA1BD91945
:10BA1800201C02F02FFCA751F8F754FB80239B0051
:10BA2800E15801204A19E250FFF7A4FEF8F748FB55
:10BA3800281CFEBD780A0020024A84239B00D058A7
:10BA48007047C046780A002010B58423134C9B0029
:10BA5800E358002B20D086239B00E1586218FF3260
:10BA680052780270E258511CFF2A01D0E15001E0DF
:10BA78000022E250F8F726FB84229200A358591EB0
:10BA8800A1500222FF32D31A3F2B02DD0220FFF71A
:10BA9800FFFDF8F715FB0123181C10BD780A0020DC
:10BAA800F7B584231F4C9B000190E058002837D03D
:10BAB8000D1E854200DD051C8626B600A159802290
:10BAC8005200571A891861180198AF420BDB2A1CDB
:10BAD80002F0D0FBA15980226B185200934200D18A
:10BAE8000023A3510AE03A1C02F0C4FB019B611C2D
:10BAF800D819EA1BFF3102F0BDFBA751F8F7E2FAAB
:10BB080084229200A1584B1BA35080225200D31AC2
:10BB18003F2B02DD0220FFF7BBFDF8F7D1FA281C06
:10BB2800FEBDC046780A002008B501200931C9B217
:10BB3800021C00F0F7FB08BD08B50020062103220F
:10BB480000F0F0FB08BD0123836070471F2201232A
:10BB58001140436083604161C360704730B51F2561
:10BB68000124294044605B0184604161FF210B404E
:10BB78000F210A401A43C460826130BDFF2352017D
:10BB88001A400F2319401143816170470223C36093
:10BB98007047006B80B27047CB43002A07D0026A17
:10BBA80013400362C162036A1943016203E0026A37
:10BBB80013400362C16270470123836042689A435D
:10BBC80042607047014B01225A60704700000240F2
:10BBD800034B012802D00122DA6000E09860704728
:10BBE80000000240034B0222012801D0DA6000E085
:10BBF8009A60704700000240034B0422012801D0DC
:10BC0800DA6000E09A60704700000240034B0822A7
:10BC1800012801D0DA6000E09A6070470000024015
:10BC2800034B8022012801D0DA6000E09A60704757
:10BC380000000240034B4022012801D0DA6000E0F6
:10BC48009A60704700000240034B012901D1186136
:10BC580000E098617047C046000002408022074B10
:10BC68005200012801D0DA6000E09A608022920038
:10BC7800012901D0DA6000E09A60704700000240B4
:10BC8800034B2022012801D0DA6000E09A60704757
:10BC980000000240C1231B061843014BD8657047BA
:10BCA80000000240E0235B051843014B58667047CB
:10BCB800000002408022074B1204012801D0DA60FC
:10BCC80000E09A608022D203012901D0DA6000E006
:10BCD8009A607047000002408022074B92030128B7
:10BCE80001D0DA6000E09A6080225203012901D075
:10BCF800DA6000E09A6070470000024007231840AD
:10BD0800024B1843024B58647047C0460000DCAC35
:10BD1800000002400F231840024B1843024B98645E
:10BD28007047C0460000C5A300000240044B102223
:10BD3800DA63D96A0722104091430843D8627047F2
:10BD480000000240054B0722D96A1040020170200A
:10BD58008143081C1043D8627047C0460000024067
:10BD680070B5094B07242040DE6A050207482140C8
:10BD780030402843D8620F20024005480901024399
:10BD8800141C0C43DC6470BD00000240FFF8FFFF88
:10BD98000000DCC370B5094B07242040DE6A0503A8
:10BDA8000748214030402843D8620F200240054808
:10BDB80009010243141C0C431C6570BD00000240BD
:10BDC800FF8FFFFF00003CDC70B5094B07242040C3
:10BDD800DE6A05040748214030402843D8620F2016
:10BDE8000240054809010243141C0C435C6570BD00
:10BDF80000000240FFFFF8FF0000CD3C034B1B6C26
:10BE08000340181A43425841C0B27047000002402C
:10BE1800044B5A6B044B13400340181A43425841D1
:10BE2800C0B2704700000240DFF00700044B9A6B75
:10BE3800044B13400340181A43425841C0B270479C
:10BE480000000240DFF00500014BD8637047C04690
:10BE580000000240044B1A6B002902D010431863FB
:10BE680001E082431A6370470000024010B50121C7
:10BE7800041C042000F0C4FB002C02D100F050FC8C
:10BE880001E000F04FFC10BD08B5002802D100F019
:10BE980047FC01E000F046FC08BD064B10B5072240
:10BEA8009C6A104004490203201C08401043986211
:10BEB80010BDC04600000240FF8FFFFF094B01285C
:10BEC80006D19A6A80201043072211400A0105E032
:10BED80007221140986A0A0180218843011C1143F6
:10BEE8009962704700000240074B9A6A012804D102
:10BEF800082002430720014003E0072001400820F2
:10BF080082431143996270470000024010B50E2128
:10BF1800041C0020012C06D1221C00F003FA201C6E
:10BF28001521221C05E0021C00F0FCF90120152156
:10BF3800002200F0F7F910BD08B5012802D113213D
:10BF4800022202E001201321002200F0EBF908BDD3
:10BF580008B5012802D11221022202E00120122193
:10BF6800002200F0DFF908BD70B5DB010C4C92012E
:10BF780003280AD81A431F2319401143A56FC60086
:10BF8800081CB0402843A06709E01A431F23194042
:10BF98000438E56F1143C00081402943E16770BD53
:10BFA80000000240072310B51A400424120122435E
:10BFB80019400902131C0B43C36010BDC368042257
:10BFC8009343C3607047026980239B001343036156
:10BFD80070470269014B134003617047FFFDFFFF83
:10BFE80003690222134303617047036902229343E2
:10BFF80003617047C36801221343C3607047C36875
:10C0080002221343C3607047026980235B00134315
:10C018000361704703690122134303617047426952
:10C0280001231A40024B1A701878C0B27047C046F4
:10C03800D802002043698B43436101624369194375
:10C04800416170474368012213434360014B032257
:10C058001A7370479C0C002008B5002A02D0FFF71D
:10C06800E9FF03E043698B434361016208BD054B67
:10C07800586A012318400840401A41424841C0B25A
:10C088007047C04600000140F7B50D1C0121009320
:10C09800041C171CFFF7EBFF0190019B0120002BEC
:10C0A80059D12D4B1A7B1E1C032A54D1002D18D1AF
:10C0B80018732A4B2A4D2363636983436361009B8A
:10C0C80020622062A762E360E3681843E060201CF6
:10C0D8000121FFF7CCFF00281DD0013D002DF6D12E
:10C0E80019E0012D24D11D731C4B23636369AB43F5
:10C0F8006361009B25622562A762E360E3681D43D4
:10C10800E560174D201C0121FFF7B1FF002802D080
:10C11800013D002DF6D1201C0121FFF7A8FF0028C2
:10C1280002D10323337316E002233373042012E091
:10C138000520022D0FD101251D73084B201C2363F8
:10C14800291C2562FFF776FF009BA762E360E3687E
:10C1580001981D43E560FEBD9C0C00205A5A5A5AAE
:10C1680001001000F8B50D1C0121161C041C1F1C31
:10C17800FFF77DFF0122002800D091E0494B197B91
:10C18800032900D08CE006991F605E609960002D3D
:10C198002DD11D732E1C434B99688E425BD2424AA7
:10C1A800079F2263616901229143616119682262D4
:10C1B800226201C9E06258681960A062E760E76816
:10C1C80004303A43394FE2605860201C0121FFF7E0
:10C1D8004EFF002802D0013F002FF6D1201C01217C
:10C1E800FFF745FF431E98412D180136D3E7012D6F
:10C1F8003BD118736369061CAB436361051C069F3A
:10C20800284BBE4227D0284A079F22636169012232
:10C218009143616119682262226201C9E06258682B
:10C228001960A062E760E76804303A431F4FE26094
:10C238005860201C0121FFF71AFF002802D0013F97
:10C24800002FF6D1201C0121FFF711FF431E984152
:10C258002D180136D3E7002D03D002221A730422C9
:10C268001EE003221A732A1C1AE00522022D17D198
:10C278000D4A187322630122226261699143616148
:10C28800226202CFE1620799A662E160E1680436A2
:10C298000A43E260069A5E60013A9A601F60021CD7
:10C2A800101CF8BD9C0C00205A5A5A5A0100100064
:10C2B80001627047014B03637047C0465A5A5A5A85
:10C2C80001230269002901D0134301E09A43131C9A
:10C2D80003617047012383607047406B7047806B30
:10C2E800704780230269002901D0134301E09A4373
:10C2F800131C036170478069034B18400840401ABB
:10C3080041424841C0B2704701070000C069044B70
:10C3180018400840401A41424841C0B27047C046E0
:10C328000107000010B5002818D11A4B0F2909D8A9
:10C338004900186803248C40A0438A40011C11431B
:10C34800196025E01039C9B24900586803248C40A7
:10C35800A0438A40011C1143596019E0012817D1F4
:10C368000C4B0F2909D84900186903248C40A043B5
:10C378008A40011C114319610AE01039C9B2490009
:10C38800586903248C40A0438A40011C1143596119
:10C3980010BDC04600800540002807D1074B01208A
:10C3A8009A688840011C1143996006E0012804D16D
:10C3B800024B88409A691043986170470080054095
:10C3C800002806D1074B01209A68884082439A606A
:10C3D80006E0012804D1034B88409A6982439A6198
:10C3E8007047C04600800540002807D1074B012050
:10C3F800DA688840011C1143D96006E0012804D19D
:10C40800024B8840DA691043D861704700800540C4
:10C41800002806D1074B0120DA6888408243DA6099
:10C4280006E0012804D1034B8840DA698243DA61C7
:10C438007047C046008005400B4901235B42CB672B
:10C448000A490B4ACB67C02149005350C221490011
:10C4580053500023191CC03189000020013350506B
:10C46800082BF7D17047C04604E100E008E100E07E
:10C4780000E100E0084BA022120508495A6000229A
:10C488009A60D9601A615A61DA611A625A620122A5
:10C4980052421A637047C04600ED00E00000FA05FA
:10C4A800024B1843024BD8607047C0460000FA059B
:10C4B80000ED00E00023037043708370C370704781
:10C4C800F0B5C17803781C4A00292AD01B49467860
:10C4D800CC68E021C900A143090A04256D1AAE40C1
:10C4E800351C0F26CE40311C8678FF240E402E4383
:10C4F80003251D409B089B00C0219B1889005F589D
:10C50800ED003601AC40AE403D1CA54334402C4301
:10C518005C5003781F205909034001209840031CF0
:10C5280006E01F205909034001209840031C2031D0
:10C5380089005350F0BDC04600E100E000ED00E086
:10C548001F23034001229A404009131C4030044A2B
:10C55800800080581840C01A43425841C0B2704702
:10C5680000E100E0024B58688002800D7047C04629
:10C5780000ED00E0014B18607047C04600EF00E096
:10C588001F234209184001238340181C6032024BC4
:10C598009200D0507047C04600E100E0024B586856
:10C5A8008005800D7047C04600ED00E0064A8023F4
:10C5B8009B00D3581F22104001228240981A434200
:10C5C8005841C0B27047C04600E100E0024B194034
:10C5D800024B08439860704780FFFF1F00ED00E0A2
:10C5E800014A024BDA6070470400FA0500ED00E0EA
:10C5F800014A024BDA6070470100FA0500ED00E0DD
:10C60800044B002901D0186102E01A6982431A61BB
:10C618007047C04600ED00E01F2318400123834007
:10C62800181C054B5A6A002902D01043586201E0D1
:10C6380082435A627047C04600ED00E070478004AC
:10C64800000F01238340181C034B5B6A0340181A30
:10C6580043425841C0B2704700ED00E0044B1F212F
:10C66800084001215A688140081C104358607047EF
:10C6780000ED00E01F21054B0840013801215A68F0
:10C688008140081C104358607047C04600ED00E028
:10C698008003000F01238340181C044B5B6A03408E
:10C6A800181A43425841C0B27047C04600ED00E036
:10C6B800014B186B7047C04600ED00E00020704742
:10C6C800024B1A69104318617047C04600ED00E03C
:10C6D800024B1A6982431A617047C04600ED00E0B8
:10C6E800024B5A69104358617047C04600ED00E09C
:10C6F800024B5A6982435A617047C04600ED00E018
:10C70800024BDA681043D8607047C04600ED00E07D
:10C71800024BDA688243DA607047C04600ED00E0F9
:10C7280030BF704720BF704740BF7047BFF36F8F5F
:10C738007047BFF34F8F7047BFF35F8F704701DFBC
:10C748007047EFF31480704780F314887047EFF355
:10C758000980704780F309887047EFF308807047B5
:10C7680080F30888704772B6704762B6704740BA5F
:10C77800704700BA7047C04670470000002804D1CF
:10C78800064B04211A688A4305E0012804D1034BAB
:10C7980004211A680A431A607047C04610E000E096
:10C7A800014B58607047C04610E000E0F8B580269D
:10C7B80084460F1C0C4B02240C4DB604002A08D0EA
:10C7C8001A68A2431A601A686E601A6814431C60DB
:10C7D80003E01A68A2431A606E603A1C0448614676
:10C7E800FFF72CFFF8BDC04610E000E000ED00E0C8
:10C7F8009AC30200024B01211A680A431A60704763
:10C8080010E000E0044B00221A605A609A60034B63
:10C81800802292045A60704710E000E000ED00E0CA
:10C82800014B98687047C04610E000E0024B80203A
:10C838001B6840021840704710E000E07047FEE7B0
:10C848007047704770477047704770477047704728
:10C858007047704770477047704770477047704718
:10C868007047704770477047704770477047704708
:10C8780070477047704770477047704770477047F8
:10C8880070477047704708B500230B4A0B499A1840
:10C898008A4204D20A49C95804331160F5E7094BA2
:10C8A800094A191D043B934203D200221A600B1C4B
:10C8B800F6E701F041FC08BD040000205800002004
:10C8C8004CE500005C000020AC0C002002B471466E
:10C8D80049084900095C49008E4402BC7047C046BB
:10C8E80003B47146490840004900095A49008E447A
:10C8F80003BC7047002934D00123002210B48842B9
:10C908002CD301242407A14204D2814202D2090176
:10C918001B01F8E7E400A14204D2814202D2490097
:10C928005B00F8E7884201D3401A1A434C08A0423A
:10C9380002D3001B5C0822438C08A04202D3001BD0
:10C948009C082243CC08A04202D3001BDC082243E7
:10C95800002803D01B0901D00909E3E7101C10BC0B
:10C968007047002801D00020C04307B4024802A144
:10C978004018029003BDC046D90000000029F0D03D
:10C9880003B5FFF7B9FF0EBC4243891A1847C046E2
:10C99800002941D010B4041C4C40A44601230022B5
:10C9A800002900D54942002800D5404288422CD3AE
:10C9B80001242407A14204D2814202D209011B01A9
:10C9C800F8E7E400A14204D2814202D249005B00A8
:10C9D800F8E7884201D3401A1A434C08A04202D310
:10C9E800001B5C0822438C08A04202D3001B9C0851
:10C9F8002243CC08A04202D3001BDC0822430028B3
:10CA080003D01B0901D00909E3E7101C6446002C78
:10CA180000D5404210BC7047002806D003DB002038
:10CA2800C043400801E08020000607B4024802A184
:10CA38004018029003BDC046190000000029EBD041
:10CA480003B5FFF7A7FF0EBC4243891A1847C04633
:10CA58007047C0468446081C6146FFE71FB500F0D2
:10CA6800E3F9002801D40021C8421FBD10B500F029
:10CA780069F94042013010BD10B500F0D5F9002821
:10CA880001DB002010BD012010BDC04610B500F02C
:10CA9800CBF9002801DD002010BD012010BDC046E3
:10CAA80010B500F079F9002801DC002010BD012044
:10CAB80010BDC04610B500F06FF9002801DA00205B
:10CAC80010BD012010BDC0469E2110B5C905041C2B
:10CAD800FFF7F0FF002803D1201C00F067FB10BD12
:10CAE8009E21C905201C00F0EBF900F05FFB8023B4
:10CAF8001B06C018F3E7C046F0B55F4656464D46DC
:10CB08004446F0B446024500C00F85B00F1C760AB3
:10CB18002D0E804641D0FF2D26D0802424040021EC
:10CB28002643F6007F3D89468B46F90F7C02780044
:10CB3800640A000E00918A463CD0FF2834D0802336
:10CB48001B041C430023E4007F380193009F4346E5
:10CB5800019A7B4049469C4611430F2900D971E050
:10CB6800764F89007F58BF46002E3ED10822022307
:10CB780091469B46D9E75A46341CC2460192019910
:10CB8800022937D0032900D1CFE0012900D0ABE03A
:10CB980053460B400022002632E0002E19D1042112
:10CBA800012289469346C0E7221C531E9A4102324D
:10CBB8000192CBE701270197002CC7D0201C01F078
:10CBC8009DFA431F9C4076235B420021181A01916D
:10CBD800BCE7301C01F092FA7625431F9E406D4257
:10CBE80000232D1A99469B469FE70C23032199465B
:10CBF8008B469AE7D446012367463B40FF2200262E
:10CC08007602D205700ADB071043184305B03CBC16
:10CC180090469946A246AB46F0BD80260023F6030F
:10CC2800FF22EDE700220026EAE78020C003064243
:10CC38003BD0044239D1061C26437602760A009B73
:10CC4800FF22DDE7281A039076016401A64239D352
:10CC5800361B1A2201230120311C5B0076000029B3
:10CC680001DBB44201D8361B0343013A002AF3DC46
:10CC7800741EA641341C1C43039A7F32002A27DD08
:10CC8800630704D00F232340042B00D0043427016A
:10CC980003D52B4B039A1C408032FE2A0BDD01235F
:10CCA80061460B40FF220026AAE706437602760A71
:10CCB8004346FF22A4E7A40101236746660AD2B2CD
:10CCC8003B409DE7039F1B22013F03970023C2E7D8
:10CCD8007E23039F5B42DB1B1B2B07DD0123614681
:10CCE8000B40002200268BE7D446C5E7221CDA4019
:10CCF800039B9E339C40231C5C1EA34113435A078D
:10CD080004D00F221A40042A00D004335F0105D54D
:10CD1800012361460B400122002671E79E0162460D
:10CD280001231340760A00226AE78026F603264389
:10CD38007602760A5346FF2262E7C04680E4000086
:10CD4800FFFFFFF74A02430270B55C0A550A430029
:10CD58004A001B0EC60F120EC90FFF2B05D0FF2A63
:10CD680008D0012093420BD070BD0120002CFBD1CC
:10CD7800FF2AF6D10120002DF6D101209342F3D1EC
:10CD8800AC42F1D18E4205D0002BEDD1201C441EBF
:10CD9800A041E9E70020E7E74A024302F0B55C0A50
:10CDA800550A43004A001B0EC60F120EC90FFF2B6F
:10CDB80031D0FF2A34D0002B16D16042604184461E
:10CDC800002A14D0002820D18E4217D1934215DCB6
:10CDD80004DBAC4212D80020AC4212D2704270413F
:10CDE8004042012318430CE0002AEDD194466F42DB
:10CDF8006F416046002805D1002FE5D0704201231D
:10CE08001843F0BD0020002FFBD148424841404262
:10CE180001231843F5E7002CCBD002204042F0E76D
:10CE2800002DC8D0F9E7C0464A024302F0B55C0AB3
:10CE3800550A43004A001B0EC60F120EC90FFF2BDE
:10CE480027D0FF2A29D0002B10D0002A15D19446CC
:10CE58006F426F416046002815D00020002F04D192
:10CE680048424841404201231843F0BD60426041B6
:10CE78008446002AECD00028F2D18E4211D07042AC
:10CE880001231843F1E7002FF7D07042012318431C
:10CE9800EBE70220002CE8D1D3E70220002DE4D1F3
:10CEA800D1E79342EBDC04DBAC42E8D80020AC428B
:10CEB800DBD270427041404201231843D5E7C04697
:10CEC800F8B5C20F430244004D024800240E161C58
:10CED8009B09000EC90FAD09FF2800D183E0012787
:10CEE80079408A425CD0221A002A00DC8EE00028B1
:10CEF8001ED1002D00D07AE0580704D00F221A4026
:10CF0800042A00D004338021C90401221940324088
:10CF180000293AD00134FF2C00D183E09B015B0A41
:10CF28005B02E4B2E405580AD20720431043F8BD77
:10CF3800FF2CE1D08021C9040D431B2A00DD31E11B
:10CF4800291C2020D140821A95406A1E95410D4324
:10CF58005B1B5801D0D59B019F09381C01F0CEF806
:10CF6800421F974094425FDC141B1F231B1B3A1C73
:10CF78009F40611C3B1CCA405F1EBB4113430024F9
:10CF8800BAE7131EB8D100230022DB08FF2C04D116
:10CF9800002B47D08020C00303435B025B0ABFE736
:10CFA800211A002944DD002827D0FF2CA4D0802096
:10CFB800C00405431B2900DDF2E0281C2027C840D7
:10CFC800791A8D40691E8D4105435B19590100D4BA
:10CFD80092E70134FF2C59D0734901221A400B40C3
:10CFE8005B08134388E7002D00D07AE777E7013A1A
:10CFF800002AADD0FF2CA0D17EE7002D00D17BE721
:10D0080001390029E1D0FF2CD4D175E7002A1BD1C2
:10D01800621CD2B2012A4BDD5F1B7A0123D5EF1ABD
:10D028000E1C9AE700237BE75F4BA41A3B4063E79B
:10D03800002946D1611CC8B2012829DDFF2924D066
:10D04800EB185B080C1C57E7002C13D0FF2818D0EE
:10D058008024E404524223431B2A4DDD0123EB1AAA
:10D06800041C0E1C75E7002F00D076E70023002271
:10D0780000248AE7002B3BD0D243002AEFD0FF28B8
:10D08800EAD12B1CFF240E1C36E7FF2400237CE783
:10D09800002C5CD1002B00D180E0002D00D12BE7C3
:10D0A8005B19580100D427E73F4A0124134023E7BE
:10D0B800002C15D1002B40D1002D63D02B1C0E1C49
:10D0C8001AE7002C21D1002B54D0C943002904D0E1
:10D0D800FF284CD01B2958DD01235B19041C75E778
:10D0E800002B19D1002D48D02B1C0E1CFF2403E760
:10D0F8002B1C041C0E1CFFE61C1C2026D440B21A54
:10D1080093405A1E93412343A9E7FF282FD0802438
:10D11800E40449422343DDE7FF24002D00D1EBE678
:10D128008022DB08D203134204D0ED08154201D156
:10D138002B1C0E1CDB00FF24DEE6002D00D1DBE6F5
:10D148005A1B500100D41CE7EB1A0E1CD4E6002B26
:10D158000DD0FF24002D00D1CEE68022DB08D203BB
:10D168001342E7D0ED081542E4D12B1CE2E72B1C53
:10D17800FF24C1E62B1C041CBEE6802300229B046E
:10D18800FF2402E7231C0022FFE61C1C2027CC40BA
:10D19800791A8B40591E8B4123439EE72B1CABE623
:10D1A800012512E70125D3E6FFFFFFFB4302590AD9
:10D1B8004300C20F1B0E00207E2B0DDD9D2B0CDCC7
:10D1C800802000040143952B0ADC9620C31AD9401D
:10D1D8004842002A00D1081C7047034BD018FBE7CF
:10D1E800963B9940F4E7C046FFFFFF7F10B5041E49
:10D1F80033D000F083FF9E231B1A962B09DC0838D6
:10D2080084406402640ADBB26402DB05600A1843E6
:10D2180010BD992B0ADD0522121A211CD1400A1CC7
:10D22800011C1B318C40611E8C411443052801DD13
:10D23800421F9440144A2240610704D00F210C4039
:10D24800042C00D0043251010AD59F23181AFF2854
:10D2580016D09401640AC3B2D6E700230024D3E7AA
:10D26800D208FF2B03D05402640ADBB2CCE7002AB1
:10D2780006D08024E40314436402640AFF23C3E74E
:10D28800FF230024C0E7C046FFFFFFFBF0B556466A
:10D2980044465F464D46F0B41F1C0B031B0B9846D3
:10D2A8004B0087B0041C81465B0DC80F161C9A46BC
:10D2B8000090002B51D06A4B9A4531D080224146CC
:10D2C80052030A43630FD2001A43664B9046002567
:10D2D800E20091469A44002402953B031B0B9B46AF
:10D2E800FD0F7B00311C5B0D019560D05C4A9342B9
:10D2F80054D08021584649030143720FC900114395
:10D30800584A8B469B18F1000020009A04436A4053
:10D3180003920F2C00D9ADE0534EA4003459A74610
:10D32800404604436ED100210225082488468946D8
:10D338000295D2E7009C0298C34649460194022808
:10D3480064D0032800D1ABE2012800D038E2019A6A
:10D35800002402400025A14660E0434623434AD00A
:10D368004046002800D1C0E100F0C8FE031E272B6C
:10D3780000DDB3E128210D1A211C083B4246E94093
:10D388009A400D1C1543221C9A40A8469146374BDB
:10D3980000251B1A9A46002402959EE75A46164312
:10D3A8000320002EB1D1B34600210220ADE75A4632
:10D3B80032431BD05B46002B00D18AE1584600F06F
:10D3C8009DFE272800DD7DE12822171A011C321C4A
:10D3D80008395B46FA408B40171C1F43331C8B40AF
:10D3E800BB46191C214B1B1A00208EE70027BB46A1
:10D3F8000021012089E70020012504248046814678
:10D4080002956AE703250C24029566E7019C0394BC
:10D41800039D01222A400024114DA146002000212D
:10D428002403260B0C0D2405114B34432D052340F2
:10D438002B435B005B08D207191C4846114307B011
:10D448003CBC90469946A246AB46F0BD00228024DB
:10D4580024039146024DE1E700240025A146DDE7BB
:10D46800FF07000001FCFFFFC0E400000DFCFFFF08
:10D47800FFFF0F805546ED1A0495D84500D953E1B2
:10D4880000D14EE1049C0025013C4E4604944746D9
:10D49800A946584603020C0E1C430902250C230416
:10D4A8001B0C0091381C291C0193FFF723FA0199E2
:10D4B80083464143381C8A46291CFFF75FFA330C20
:10D4C800090419438A450CD95B460919013B8C426A
:10D4D80000D947E18A4500D844E1022252429344E8
:10D4E80009195346CB1A181C291C9846FFF702FA4B
:10D4F800071C0198291C784382464046FFF73EFAEC
:10D5080036040B04360C33439A4509D91B197A1E85
:10D518009C4200D924E19A4500D821E1023F1B1919
:10D528005E4632041743380CBB46009E009F5146A6
:10D538003F0C32045B1A5946BA46120C0F043F0CD2
:10D54800904651467A434F434146414356467043BD
:10D55800CF19160CBE19B14202D980277F02C01913
:10D56800310C12043604120C4018B618834200D24B
:10D57800C4E000D1BEE0191A4846861BB145BF4138
:10D588007F42CF1BA74200D113E1291C381CFFF7AB
:10D59800B1F9019902904143381C8946291CFFF7CB
:10D5A800EDF9330C0904194389450CD9029B091973
:10D5B800013B8C4200D9FFE0894500D8FCE0029F7E
:10D5C8000919023F02974F46CF1B381C291C0597A3
:10D5D800FFF790F9071C0198291C784381460598A4
:10D5E800FFF7CCF936040904360C0E43B14509D9C6
:10D5F80036197B1EB44200D9E0E0B14500D8DDE021
:10D60800023F3619029D4946761A290439430B040C
:10D6180057460A0C1B0C40464546584355437B4326
:10D628007A43EB18070CDB199D4202D980256D025D
:10D6380052191D0C00041B04000C52191B189642A9
:10D6480035D300D1FCE001231943049E994FF51905
:10D65800002D00DCA1E0480709D00F230B40042B64
:10D6680005D00B1D8B42894149428B44191C5A46EF
:10D67800D20107D5904B5C46049E80271C40FF00D2
:10D68800A346F5198D4B9D427ADD039C0122224069
:10D6980000248B4DA146C1E6802424034746274237
:10D6A8004CD13C432403240B009A854DB6E6361929
:10D6B800481EB4425ED9011C9642C4D1009E9E42C7
:10D6C800C1D1C2E7031C283B311C99408B4600217D
:10D6D80088E6301C00F012FD203072E6283B211C41
:10D6E800994000228846914651E6201C00F006FD2C
:10D6F80020303BE60021B14500D33DE7009F5A4664
:10D70800B944B945BF417F423F19FB18013A9C42D1
:10D718001ED2984200D97EE000D1B5E0191A93468E
:10D728002AE7894500D8ADE6484646464246770886
:10D73800D3074608C0071E438146AAE6584620423A
:10D7480012D1044324032A1C240B89465C4D65E648
:10D75800A342E3D1009F4F45DBD9211A93460BE73B
:10D76800171CDDE69B46BCE63C432403240B009AC9
:10D77800534D53E6B24259D800D18AE0011C62E702
:10D788005F46C9087B07039E0B437C026D05012297
:10D798009946240B6D0D324040E64A4B049FDB1B33
:10D7A800382B10DD039C0122224000240025A146CD
:10D7B80034E60121494248E7029304E71F1C21E7A8
:10D7C800019C039441E71F2B40DC3F48049F0C1C3D
:10D7D8003A1858469140DC40904020430A1C511E9C
:10D7E8008A41011C11435A46DA40131C480709D0E4
:10D7F8000F220A40042A05D00A1D8A42894149425B
:10D808005B18111C1A0234D5039C01222240002403
:10D818000125A14602E6009F02214942B9448B44F2
:10D82800B945894149420919CB18A4E6009D881ECB
:10D838006900A942AD416D422C19361900913AE7A9
:10D84800002B00D033E70024009437E71F4A049CDC
:10D858005D46121BD5402A1C202B1FD01C4E5F464C
:10D86800A3199F403B1C19434B1E994111430023A8
:10D87800BCE75A07C9080A43039F91465B02012285
:10D888001C0B3A400025C9E54E45C4D893460021F3
:10D8980072E6009F9F42C9D3011C0FE70023E2E70D
:10D8A800802424035F463C432403240B019A8946C1
:10D8B800034DB3E5FF030000FFFFFFFEFE07000076
:10D8C800FF07000002FCFFFF1E040000E2FBFFFF51
:10D8D8003E040000F0B5564644465F464D46F0B457
:10D8E8001F1C0B031B0B9A464B0087B0041C804679
:10D8F8005B0DC80F161C02938146002B68D0694B3C
:10D908000299994232D08022534652031A43D200D8
:10D91800630F1A439246644AE000891880460291D0
:10D92800002400253B031B0B9B467800FB0F321C91
:10D93800400D039300D175E05A4B984269D080227C
:10D94800594652030A43730FD2001A43564B934663
:10D95800C018F200002303994E4671401C430F2C57
:10D9680000D9A9E0514EA4003459A74653461C4398
:10D9780000D087E00025AA46A84608240225D1E75A
:10D988004946022D6CD0032D00D117E2012D00D09D
:10D9980058E10D40EDB20024A9460023A04600201E
:10D9A800002125030A0D1C052D0B1205404B2A43A7
:10D9B800134023435B004C465B08E207191C4046B2
:10D9C800114307B03CBC90469946A246AB46F0BD11
:10D9D8005346234350D05346002B00D184E1504690
:10D9E80000F08CFB031E272B00DD76E128210D1AA1
:10D9F800211C083B5246E9409A400D1C1543221C45
:10DA08009A40AA4690462B4B00241B1A02930025E5
:10DA180088E75B461E430323002E9CD1B3460022B1
:10DA2800022398E75B46334321D05846002800D1AB
:10DA38004EE100F063FB272800DD42E128210F1AA0
:10DA4800021C311C083A5B46F94093400F1C1F43E7
:10DA5800331C9340BB461A1C164B181A00237AE74E
:10DA680001230B4000249946A0460E4B97E7002758
:10DA7800BB46002201236EE7002104248A4688461B
:10DA880001254FE70C2403254CE700258024A946EF
:10DA98002403A846034B82E7DA46904603991D1CE7
:10DAA8006FE7C046FF07000001FCFFFF00E500002C
:10DAB800FFFF0F800DFCFFFF029F160C3818049023
:10DAC8004046070C0004000C1204120C031C5343BC
:10DAD800041C3D1C7443554398463B1C734364190E
:10DAE800A44644460293230C63449D4204D9029DF4
:10DAF800802464022D1902951D0C039545462C04BB
:10DB08001B04240C1C1905945C46230C051C584363
:10DB18002404240C8446381C604365435F438146D3
:10DB2800CC44280C6044BB46814502D980277F023B
:10DB3800BB442D04070C2D0C000440195546BC4667
:10DB48002F04E3448446280C3D0C2F1C5743B84649
:10DB58002F1C77434243B94647463F0C9144BA4687
:10DB6800D14446434A4502D980225202B6184F464C
:10DB78003A0CB6183A0447463F043F0CB8462F1CE7
:10DB880067435D434443584365190190380C2D1889
:10DB98004244B846AC4204D9019880235B02C018BD
:10DBA8000190039C029F201C6044C0196045A44159
:10DBB80047466442A4462B043C049946240C4C4432
:10DBC800A046D8448018C246E24490429241574643
:10DBD80052429146F219E245BF417F424B46BC464C
:10DBE800D845BF41D4187F4263461F432D0C7F1987
:10DBF800B24292414C45AD4152426D421543019E9D
:10DC08007D19AB19E20D5B02059F134342023A43AB
:10DC18009A46531E9A41C30D101C184364022043B0
:10DC280080465046C0010DD5454601225646049C03
:10DC38006B082A401A43F30701341A437608049400
:10DC48009046B246049E634FF319002B61DD4046AF
:10DC580040070BD00F2244462240042A06D04246F1
:10DC68000432424580414042824490465546ED0187
:10DC780007D5594B5646049F80201E40C000B24627
:10DC88003B18564A934200DDEAE644465546E20808
:10DC98006807104301226C025B050A408046240B8A
:10DCA8005B0D91467BE6DA4690461D1C69E68024AA
:10DCB8002403574627421CD13C432403240B484BDA
:10DCC8006DE6031C283B311C99408B460022C3E6B5
:10DCD800301C00F013FA2030ADE6283B211C994097
:10DCE80000228A4690468EE6201C00F007FA203073
:10DCF80078E65846204207D1044303992403240BAD
:10DD080089469046364B4AE63C432403240B344B61
:10DD180045E6344B049E9B1B382B06DD01230B4044
:10DD280000249946A046002339E61F2B25DC049CD5
:10DD38002D4D46466019524644468640DC40824096
:10DD48005746301C2243DF40441EA04102433B1C7F
:10DD5800540709D00F201040042805D0101D904208
:10DD6800924152429B18021C1D021AD501230B40F6
:10DD780000249946A046012311E61C48049C5546F8
:10DD8800001BC540281C202B16D0194E5746A21937
:10DD980097403A1C43461A43531E9A4102430023B4
:10DDA800D6E758075B02D2081C0B01230B4010432F
:10DDB800994680460023F2E50022EBE780242403FD
:10DDC80050460123044319402403240B8946044B7D
:10DDD800E5E5C046FF030000FFFFFFFEFE07000069
:10DDE800FF07000002FCFFFF1E040000E2FBFFFF2C
:10DDF8003E04000070B50B1C124C09030E0B5900B1
:10DE0800021C490DDD0F0020A14211DD0E488142A0
:10DE18000FDC8020400306430C48401A1F280BDD06
:10DE28000B4A521AD640321C5042002D00D1101C09
:10DE380070BD084BE818FBE7074BC240C9188E4075
:10DE48003243F1E7FE0300001D0400003304000024
:10DE580013040000FFFFFF7FEDFBFFFFF8B5041E72
:10DE680031D0C70F00D04442201C00F047F9184DAC
:10DE78002D1A0A2819DD0B38844024036D05240B5C
:10DE88006D0D3A1C0026002000210B0D2403240BE5
:10DE98001B0523430F4C2D051C402C4364006408CC
:10DEA800D307211C301C1943F8BD061C1536231C4A
:10DEB800B3401E1C0B23181AC44024036D05240B01
:10DEC8006D0D3A1CDFE70022002500240026DAE762
:10DED8001E040000FFFF0F8010B5041E28D000F0BC
:10DEE8000DF9154A121A0A2815DD0B388440240347
:10DEF8005205240B520D0023002000212403181C76
:10DF08000B0D240B1B0523430C4C12051C4014431A
:10DF18006400610810BD031C1533211C99400B1CBB
:10DF28000B21081AC44024035205240B520DE3E7C1
:10DF3800002200240023DFE71E040000FFFF0F80FB
:10DF480043001B0E5A1C4102D2B270B54C0AC50FD1
:10DF5800012A17DDE02292006407090B98180022B5
:10DF680000231E0D221C34050C431B4940054008A4
:10DF78002140014349004908ED070B1C2B43101CA5
:10DF8800191C70BD002B15D1002C1CD0201C00F0D2
:10DF9800B5F80A281ADC0B21091A231CCB40191CD6
:10DFA800031C15339C400D4B0903181A4005090B37
:10DFB800400DD4E7002C03D06407090B0848CEE7CE
:10DFC80007480021CBE700200021C8E7011C0B39D6
:10DFD8008C40211C0024E6E7FFFF0F808903000026
:10DFE800FF070000F0B54B000D03420F5B0D6D0AF3
:10DFF80015435A1C5205CC0FC600520D012A27DDC5
:10E00800394FDA19FE2A1ADC002A35DD8001ED00C5
:10E01800431E98412843760F3043430704D00F230B
:10E028000340042B00D004308021C904014027D0CC
:10E038000132FF2A1DD083015B0AD1B201E0FF2122
:10E0480000235802C905400AE40708432043F0BDED
:10E05800002B06D1354311D10021002043025B0A71
:10E06800EFE72E43EBD08020ED0080042843FF2209
:10E07800D3E7FF210023E4E717320DDA0520002259
:10E08800C008D1B2FF2AE9D10028D9D08023DB0308
:10E0980003435B025B0AD4E7802214491204154348
:10E0A800C91A1F290DDC124A371C9B18281C9F40CF
:10E0B80098403B1C5A1E93411843CE4030430022DF
:10E0C800ABE70C4F2A1CFF1AFA40171C202909D06D
:10E0D800094A98188540281C3043461EB0413843E9
:10E0E80000229AE70020F7E780FCFFFF9E0300006C
:10E0F80082FCFFFF7E030000A2FCFFFF1C2101231E
:10E108001B04984201D3000C10391B0A984201D312
:10E11800000A08391B09984201D30009043902A2F0
:10E12800105C40187047C046040302020101010157
:10E13800000000000000000038B5434D04232B61A7
:10E148008D22424B9201DA6080231B04AB606A6B1C
:10E1580001243D4B2242FAD03D4A3E489A623E4A4B
:10E16800DC625A643D4A00219A6462421A61FDF7F2
:10E1780069FF3848211CFEF7B4F8E2200001FDF7DA
:10E1880089FD201CFDF74CFD2B6C80221342FBD02F
:10E19800304B042019690A431A61FDF7C7FD0020B6
:10E1A800FDF77BFE284B5B6B5A060BD42C48FDF71A
:10E1B80079FD0120FDF73EFD6A6B40231A42FBD032
:10E1C800214AD3630320FEF76BF9F5F781FFF6F7D1
:10E1D80035F9FCF7B8FD23498023DB04CB67224AD5
:10E1E800C021490053501360F6F7E0F8FAF7F6F942
:10E1F800F9F767FFFCF738FAF6F7F8F81B4CE08CEC
:10E20800F6F780F82078FAF741F8E078FAF7A8F8F6
:10E218006079A1682269FAF7B3F8FAF761FCFCF7AC
:10E2280063F9FCF7E3FAF9F7E9F8FAF773FAF9F79B
:10E23800D5F9FAF779FFFAF76EFA0D4B1B78002B30
:10E24800F5D0002038BDC046000002400000034061
:10E258002C080000000001400000DCAC0000C5A351
:10E26800280E000004E100E000E100E008000020C2
:10E2780068090020F0B50F2A35D9031C0B439C0709
:10E2880035D1161C103E36093501451910350C1CC0
:10E29800031C27681F6067685F60A7689F60E7685E
:10E2A8001034DF601033AB42F3D1731C1B01C51867
:10E2B800C9180F231340032B1BD91C1FA4080134B2
:10E2C800A4000023CE58EE500433A342FAD1ED182F
:10E2D800C91803231A4005D00023CC5CEC54013341
:10E2E8009342FAD1F0BD051C002AF5D1FAE7051CC6
:10E2F800F2E71A1CF8E7C046F401000064000000C9
:10E308000180080800000000006400000000000010
:10E3180000000000C800000000000000000000002D
:10E32800010003E80000000000000003E80000000E
:10E3380000000200FA060003000000000037060093
:10E34800000000000000000004010000AD00000013
:10E358008200000057000000410000002B00000070
:10E3680021000000160000000B000000120110013F
:10E3780002000010D0165306000101020301090231
:10E388004300020100C0320904000001020201003A
:10E3980005240010010524010101042402060524B6
:10E3A8000600010705830310000109040100020AA1
:10E3B8000000000705810240000007050202400036
:10E3C800000000005EE400002EE4000004E4000009
:10E3D800F0E3000000000000000000000000000062
:10E3E8000000000000000000140354004D0043002A
:10E3F8004D002D0031003100310030002A03540057
:10E408004D0043004D002D00310031003100300037
:10E418002000730074006500700052006F006300F4
:10E428006B006500720030035400720069006E00D2
:10E4380061006D006900630020004D006F007400EA
:10E4480069006F006E00200043006F006E007400CA
:10E4580072006F006C000403090400001000000043
:10E468004000000040000000100000001000000004
:10E4780000000000000000004CCC0000FECB0000B3
:10E488002CCC000086CB00002CCC000022CC000055
:10E498002CCC000086CB0000FECB0000FECB000099
:10E4A80022CC000086CB00007ECB00007ECB000093
:10E4B8007ECB000032CC00007CD4000018D40000D1
:10E4C80060D4000046D3000060D4000054D400009B
:10E4D80060D4000046D3000018D4000018D400000F
:10E4E80054D4000046D300003CD300003CD30000C5
:10E4F8003CD30000A0D60000C0DA0000AEDC00006B
:10E50800AEDC0000A0DA00008AD900008AD9000039
:10E5180092DA0000A0DA00008AD9000092DA00003E
:10E528008AD90000A0DA000088D9000088D9000044
:10E5380088D90000B6DC000031313130563130382E
:04E5480000000000CF
:10E54C0040E500000001020000080000010000008E
:10E55C0002000000000000000000000000000000AD
:10E56C000000000000000000000007000000000098
:10E57C00000000000000000000000000000000008F
:10E58C0000000000FFFFFFFFA120000000000200C0
:04E59C00000000007B
:04000003000040C8F1
:00000001FF
